:100000000C9426040C9443040C9443040C940C2A82
:100010000C949E320C9443040C9443040C944304BB
:100020000C9443040C9443040C9443040C94D01695
:100030000C9443040C9443040C9443040C94430424
:100040000C94B1190C9443040C9460140C94221475
:100050000C9443040C9443040C9443040C94430404
:100060000C9443040C944304490B2D132D13530B90
:10007000600B6D0B7A0B2D137E0B2D138C0B2D1338
:10008000960BA00BD10B2D132D132D13AA0BB70B11
:10009000C40BF111021221120212251238122B1276
:1000A00031124D125312621279129D12A712B3121D
:1000B000BD12622368236B236E2373237B23852366
:1000C000F123F123F1238D2390239923A223F123FC
:1000D000F123F123F123F123F123AA23B423C02335
:1000E000C823CB23D423DD23E323FD2D002E052EAF
:1000F000082E0B2E0E2E112E142E172E1A2E1D2EFC
:10010000292E292E292E292E292E292E292E292E37
:10011000232E202E262E702E732E762E792E7C2EB8
:100120007F2E822E852E084AD73B3BCE016E84BCA3
:10013000BFFDC12F3D6C74319ABD56833DDA3D0041
:10014000C77F11BED9E4BB4C3E916BAAAABE00008A
:1001500000803F05A84CCDB2D44EB93836A9020C68
:1001600050B9918688083CA6AAAA2ABE0000008041
:100170003F003E0D0A002C4C696D3A002C52583A53
:10018000002C4275663A002C002C57506F733A00D1
:100190002C002C4D506F733A003C446F6F72003C42
:1001A000436865636B003C416C61726D003C486F55
:1001B0006D65003C486F6C64003C52756E003C49B4
:1001C000646C65005D0D0A005B302E396A2E32309A
:1001D0003136303331373A000D0A003D00244E00ED
:1001E0005D0D0A00205300204600205400204D38A9
:1001F00000204D3900204D3500204D3400204D3376
:1002000000204D3200204D3100204D300020473974
:100210003400204739330020473931002047393036
:10022000002047323000204732310020473139006A
:100230002047313800204731370020470047333806
:100240002E0047383000473300473200473100471F
:1002500030005B005D0D0A005B544C4F3A005D0DB1
:100260000A002C005B4739323A005D0D0A002C0071
:100270003A003330003238005B47005D0D0A003A27
:10028000002C005B5052423A00290D0A00206D619B
:10029000782074726176656C2C206D6D002061632E
:1002A00063656C2C206D6D2F7365635E3200206D6D
:1002B000617820726174652C206D6D2F6D696E0000
:1002C0002C20737465702F6D6D007A0079007800B2
:1002D0002028003D0024002028686F6D696E67208B
:1002E00070756C6C2D6F66662C206D6D290D0A0083
:1002F0002028686F6D696E67206465626F756E6334
:10030000652C206D736563290D0A2432373D00206A
:1003100028686F6D696E67207365656B2C206D6D45
:100320002F6D696E290D0A2432363D002028686F32
:100330006D696E6720666565642C206D6D2F6D6933
:100340006E290D0A2432353D00290D0A2432343D30
:10035000002028686F6D696E672064697220696E7D
:1003600076657274206D61736B3A002028686F6D3A
:10037000696E67206379636C652C20626F6F6C29EE
:100380000D0A2432333D00202868617264206C69B4
:100390006D6974732C20626F6F6C290D0A243232E0
:1003A0003D002028736F6674206C696D6974732C2E
:1003B00020626F6F6C290D0A2432313D00202872B3
:1003C00065706F727420696E636865732C20626F4C
:1003D0006F6C290D0A2432303D00202861726320A1
:1003E000746F6C6572616E63652C206D6D290D0AEA
:1003F0002431333D0020286A756E6374696F6E2066
:10040000646576696174696F6E2C206D6D290D0AC3
:100410002431323D00290D0A2431313D002028735A
:100420007461747573207265706F7274206D61737E
:100430006B3A00202870726F62652070696E2069C7
:100440006E766572742C20626F6F6C290D0A2431F0
:10045000303D0020286C696D69742070696E7320CE
:10046000696E766572742C20626F6F6C290D0A2498
:10047000363D0020287374657020656E61626C657E
:1004800020696E766572742C20626F6F6C290D0A7C
:1004900024353D00290D0A24343D0020286469726A
:1004A00020706F727420696E76657274206D61734E
:1004B0006B3A00290D0A24333D00202873746570BF
:1004C00020706F727420696E76657274206D61732E
:1004D0006B3A002028737465702069646C65206431
:1004E000656C61792C206D736563290D0A24323D9A
:1004F000002028737465702070756C73652C2075EE
:10050000736563290D0A24313D0024303D00242405
:10051000202876696577204772626C207365747451
:10052000696E6773290D0A24232028766965772070
:100530002320706172616D6574657273290D0A24E0
:100540004720287669657720706172736572207321
:1005500074617465290D0A2449202876696577201D
:100560006275696C6420696E666F290D0A244E20DD
:100570002876696577207374617274757020626C77
:100580006F636B73290D0A24783D76616C75652065
:100590002873617665204772626C20736574746994
:1005A0006E67290D0A244E783D6C696E65202873AC
:1005B000617665207374617274757020626C6F630C
:1005C0006B290D0A24432028636865636B206763E9
:1005D0006F6465206D6F6465290D0A245820286BAF
:1005E000696C6C20616C61726D206C6F636B290D9E
:1005F0000A2448202872756E20686F6D696E672026
:100600006379636C65290D0A7E20286379636C65C4
:10061000207374617274290D0A212028666565644F
:1006200020686F6C64290D0A3F202863757272651B
:100630006E7420737461747573290D0A6374726C1F
:100640002D7820287265736574204772626C290DBD
:100650000A000D0A4772626C20302E396A205B272F
:10066000242720666F722068656C705D0D0A005D3E
:100670000D0A00526573746F72696E672064656657
:1006800061756C74730050676D20456E640043683B
:1006900065636B20446F6F720044697361626C65BF
:1006A0006400456E61626C65640043617574696FD6
:1006B0006E3A20556E6C6F636B6564002724482783
:1006C0007C2724582720746F20756E6C6F636B0035
:1006D000526573657420746F20636F6E74696E75F4
:1006E00065005B000D0A00486F6D696E67206661EA
:1006F000696C0050726F6265206661696C004162CE
:100700006F727420647572696E67206379636C65BB
:1007100000536F6674206C696D697400486172647F
:10072000206C696D697400414C41524D3A20000DB6
:100730000A00496E76616C69642067636F646520A6
:1007400049443A00556E646566696E656420666565
:100750006564207261746500556E737570706F7298
:1007600074656420636F6D6D616E64004D6F6461CC
:100770006C2067726F75702076696F6C6174696F39
:100780006E004C696E65206F766572666C6F7700DF
:10079000486F6D696E67206E6F7420656E61626C64
:1007A000656400416C61726D206C6F636B004E6F0D
:1007B000742069646C6500454550524F4D20726548
:1007C0006164206661696C2E205573696E672064D0
:1007D000656661756C74730056616C7565203C20AC
:1007E0003320757365630053657474696E672064A4
:1007F000697361626C65640056616C7565203C20AC
:100800003000496E76616C69642073746174656D43
:10081000656E7400426164206E756D62657220665B
:100820006F726D61740045787065637465642063F0
:100830006F6D6D616E64206C6574746572006572B5
:10084000726F723A20006F6B0D0A000011241FBEF8
:10085000CFEFD8E0DEBFCDBF11E0A0E0B1E0E6ED24
:10086000F1E702C005900D92A430B107D9F726E058
:10087000A4E0B1E001C01D92A23DB207E1F70E94E1
:1008800045040C94E9380C9400008CE38AB98FE09D
:1008900087B90E94F0130E94FD230E942C1A0E9427
:1008A00091328EE1EBE2F5E0DF011D928A95E9F7E6
:1008B00081E080932B0578948091C10684FF03C06A
:1008C00081E080932C050E94BE140E940C090E94B6
:1008D00059130E94C8130E94BB290E94B32D0E9485
:1008E0003B250E94001A0E948B280E941E0910922C
:1008F0002B051092490510924B0510922D05109270
:100900002E050E94F215DFCFEF92FF921F93CF9337
:10091000DF9300D000D0CDB7DEB77C01122F8091DD
:10092000C10685FF0BC0C70149835A836B837C8353
:100930000E94172C7C816B815A81498180912C0502
:10094000823031F149835A836B837C830E94C314C4
:1009500080912B0581111CC00E948A2549815A81F2
:100960006B817C81882339F00E94E91549815A8185
:100970006B817C81E7CF212FC7010F900F900F90E3
:100980000F90DF91CF911F91FF90EF900C949225E3
:100990000F900F900F900F90DF91CF911F91FF90CC
:1009A000EF9008952F923F924F925F926F927F92B5
:1009B0008F929F92AF92BF92CF92DF92EF92FF926F
:1009C0000F931F93CF93DF93CDB7DEB7E7970FB6A3
:1009D000F894DEBF0FBECDBF9C8B8B8B1B013A0101
:1009E00009871A872B873C87AF8A2D961FAD2D97D5
:1009F0002E962FAD2E97298B2F963FAD2F973D8B9F
:100A000084E0889EA00111245A834983AB89BC8964
:100A1000A40FB51FB98FA88F460D571D5B8F4A8F46
:100A2000FA0180809180A280B3802D913D914D91FB
:100A30005C91C501B4010E9497346C8F7D8F8E8FBD
:100A40009F8FF4E01F9F800111242B893C89200F88
:100A5000311F39A328A3A301400F511F5BA34AA351
:100A6000DA014D905D906D907C90F901208131818B
:100A700042815381C301B2010E9497346CA37DA3CC
:100A80008EA39FA3A501940150582D873E874F87C1
:100A9000588BD301C201B0588D839E83AF83B88732
:100AA000E981FA81E20DF31D2C8D3D8D4E8D5F8D18
:100AB00060817181828193810E9496342B013C0177
:100AC000F101E00FF11F2CA13DA14EA15FA16081BA
:100AD0007181828193810E9496344B015C01A30154
:100AE00092016D857E858F8598890E94AE376983D6
:100AF0007A838B839C83A50194016D817E818F8194
:100B000098850E94AE379B01AC0169817A818B8107
:100B10009C810E94973469837A838B839C83A5018F
:100B200094016D857E858F8598890E94AE374B0133
:100B30005C01A30192016D817E818F8198850E9465
:100B4000AE379B01AC01C501B4010E9496342981E6
:100B50003A814B815C810E940A352B013C019D89C1
:100B6000992399F02DEB37E346E055EBC301B20131
:100B70000E94733787FD1DC02BED3FE049EC50E428
:100B8000C301B2010E94963412C02DEB37E346E058
:100B900055E3C301B2010E947035181654F02BEDD5
:100BA0003FE049EC50E4C301B2010E9497342B01AD
:100BB0003C018090BD069090BE06A090BF06B0900C
:100BC000C00629853A854B855C85CA01B9010E941A
:100BD0009734A50194010E9496349B01AC01C50194
:100BE000B4010E94AE370E943B384B015C0120E00B
:100BF00030E040E05FE3C301B2010E94AE372985D7
:100C00003A854B855C850E94AE379F77A50194019C
:100C10000E9477350E944D360E94E4357E8B6D8BA5
:100C2000DB01AB2B09F486C14B01A12CB12CBF8990
:100C3000BB2361F0C501B4010E9410369B01AC01D9
:100C4000C701B6010E94AE376B017C01C501B4013A
:100C50000E9410364B015C019B01AC01C301B20143
:100C60000E94773569877A878B879C87F989E4E0CA
:100C7000FE9FC00111242B893C89280F391F3A8B14
:100C8000298BF101E80FF91FD9012D913D914D916B
:100C90005C9160817181828193810E949634A5016B
:100CA00094010E9477356CAB7DAB8EAB9FAB2985F1
:100CB0003A854B855C85CA01B9010E94AE379B011C
:100CC000AC0160E070E080E090E40E9496344B015B
:100CD0005C012BEA3AEA4AE25EE369857A858B8514
:100CE0009C850E94AE372B013C0120E030E040E8BB
:100CF00050E4C501B4010E9497349B01AC01C301CB
:100D0000B2010E94AE3768A779A78AA79BA720E007
:100D100030E040E05FE3C501B4010E94AE376CA74C
:100D20007DA78EA79FA7198201E010E0ED89FE89BB
:100D30000E171F0709F4FEC0B981BC3008F04AC085
:100D40002CA53DA54EA55FA56D817E818F819885DF
:100D50000E94AE374B015C0128A539A54AA55BA5C9
:100D60006D857E858F8598890E94AE37A501940197
:100D70000E949734B62EA72E982E892E2CA53DA51D
:100D80004EA55FA56D857E858F8598890E94AE37BB
:100D90002B013C0128A539A54AA55BA56D817E8163
:100DA0008F8198850E94AE379B01AC01C301B201CF
:100DB0000E9496346D877E878F87988BE981EF5FDD
:100DC000E9838B2D9A2DA92DB82D8D839E83AF831A
:100DD000B8876EC0B80180E090E00E941036298587
:100DE0003A854B855C850E94AE374B015C010E94C1
:100DF00074356D837E838F839887C501B4010E940B
:100E000031384B015C01EA8DFB8D80819181A2819B
:100E1000B3819C01AD01505829833A834B835C8395
:100E2000AAA1BBA18D919D910D90BC91A02D88ABE5
:100E300099ABAAABBBAB2D813E814F8158856981AF
:100E40007A818B819C810E94AE372B013C01A501E8
:100E5000940168A979A98AA99BA90E94AE379B0130
:100E6000AC01C301B2010E9497346D877E878F87E2
:100E7000988BA501940169817A818B819C810E9464
:100E8000AE374B015C012D813E814F81588568A9A9
:100E900079A98AA99BA90E94AE379B01AC01C50123
:100EA000B4010E9496346D837E838F839887198264
:100EB0002D853E854F8558896C8D7D8D8E8D9F8DBE
:100EC0000E949734E88DF98D6083718382839383C8
:100ED0002D813E814F8158856CA17DA18EA19FA15E
:100EE0000E949734A8A1B9A16D937D938D939C9393
:100EF00013972CA93DA94EA95FA9E989FA896081B8
:100F00007181828193810E949734A989BA896D93F6
:100F10007D938D939C9313972F89B701A6018B899D
:100F20009C890E94840480912B05811121C00F5F50
:100F30001F4FFCCE2F89B701A601C101E7960FB65E
:100F4000F894DEBF0FBECDBFDF91CF911F910F91FF
:100F5000FF90EF90DF90CF90BF90AF909F908F90D9
:100F60007F906F905F904F903F902F900C948404EF
:100F7000E7960FB6F894DEBF0FBECDBFDF91CF91DD
:100F80001F910F91FF90EF90DF90CF90BF90AF90A7
:100F90009F908F907F906F905F904F903F902F9099
:100FA00008958F929F92AF92BF92CF92DF92EF926D
:100FB000FF924B015C0180912C05823009F447C0FF
:100FC00020E030E040EA51E4C501B4010E94AE37B0
:100FD0000E944D360E94E4356B017C010E9474161C
:100FE00020E030E04AE754E4C501B4010E94AE3786
:100FF0004B015C0182E38C9DB0018D9D700D11242D
:1010000080E090E00E9410369B01AC01C501B40164
:101010000E9496340E944D360E94E435CB010E9416
:101020007F29C114D10499F00E94C31421E0C21A8F
:10103000D10880912B0581110AC08FEF90E722E043
:10104000815090402040E1F700C00000EACFFF90BF
:10105000EF90DF90CF90BF90AF909F908F900895CA
:101060000E94B02984E00E94402A83E00E94402A26
:101070000E94C31480912B05811104C00E941E0997
:101080000C94BB290895CF92DF92EF920F93CF93E8
:10109000DF9300D000D01F92CDB7DEB76C018091F6
:1010A0002C05823009F481C02D8349835A836B83D8
:1010B0007C830E94741610924705802F0E94B62DE3
:1010C0000E94C82D2D8149815A816B817C818823A2
:1010D000A1F09FB7F89480914B05806180934B05F8
:1010E0009FBF2D8349835A836B837C830E94C314E3
:1010F0007C816B815A8149812D8180912B058111E1
:1011000054C0C6010E94840481E080934A059FB7C1
:10111000F894809149058260809349059FBF0E94A1
:10112000C31480912B05811140C080912C05811141
:10113000F6CF80914A058130A9F4EE2051F08CE081
:10114000EFE2F5E0ABE3B5E001900D928A95E1F7AF
:101150000CC09FB7F89480914B05806180934B053C
:101160009FBF03C081E08093470510924A050E940B
:10117000C31480912B05811118C00E94001A0E948F
:101180003B250E948B286FE275E0C6010E947C34EB
:101190000F900F900F900F900F90DF91CF910F91C4
:1011A000EF90DF90CF900C94F72F0F900F900F904F
:1011B0000F900F90DF91CF910F91EF90DF90CF9034
:1011C00008958091490584FD26C09FB7F8948091C9
:1011D00049058061809349059FBF0E945F130E946B
:1011E000C61380912C05982F9C7021F490912D05A9
:1011F000913089F49FB7843029F4F89480914B059D
:10120000806204C0F89480914B05886080934B0500
:101210009FBF0C94A51608958FE3ECE4F5E0DF0181
:101220001D928A95E9F76FE675E080E00E94C22280
:10123000811103C087E00C94E72D08956FE275E0FB
:1012400083E695E00C947C342F923F924F925F920C
:101250006F927F928F929F92AF92BF92CF92DF92C6
:10126000EF92FF920F931F93CF93DF93CDB7DEB72B
:10127000AB970FB6F894DEBF0FBECDBF98A38F8F8C
:1012800089E3EBE8F5E0DF011D928A95E9F78AE052
:10129000ECE4F5E0ACE8B5E001900D928A95E1F759
:1012A0001D8E212C312CA12CB12C19A2512C1E8E5B
:1012B00066246394712C08E0402E9924939485E071
:1012C000882E8D8DEF8DF8A1E80FF11D0081002390
:1012D00009F48AC29FEB900F9A3110F00C941F13FF
:1012E0008F5F8D8FAE01475E5F4FBE01635E7F4FA4
:1012F0008F8D98A10E94CD28882311F40C9421137E
:10130000C98CDA8CEB8CFC8CC701B6010E947C384E
:101310000E94E435162F70E080E090E00E941236C3
:101320009B01AC01C701B6010E94963420E030E079
:1013300048EC52E40E94AE370E9411380E94E43516
:10134000073421F00D3409F450C192C1183209F468
:1013500032C1E8F4143160F4113108F0D7C0143010
:1013600009F45AC008F48EC01A30D9F10C942D1328
:101370001C31B9F128F4163108F4F7C00C942D1380
:101380001E3179F1163209F47DC00C942D131D33F2
:1013900009F40BC1A8F4153309F461C040F41B3201
:1013A00009F4ECC0113309F4E9C00C942D131C337B
:1013B00010F00C942D1316531093920589E000C180
:1013C0001C3540F41A3508F0B0C0103509F49BC044
:1013D0000C942D131C3529F01F3508F4BDC00C9456
:1013E0002D136115710531F4BE8DB1110C942313C9
:1013F000E1E0EE8F1C3199F038F4143069F01A30C6
:1014000009F0DBC082E02CC0153349F11C3559F1DD
:101410001E3109F0D2C013C090928B05CEC0611569
:10142000710549F06A30710511F00C942D1324E018
:1014300020938B0509C0F3E0F0938B0505C061157F
:10144000710521F480928B0580E0BFC06A30710580
:1014500011F00C942D1336E030938B05F5CF87E017
:1014600080938B05AAC06115710549F06A3071053A
:1014700011F00C942D1399E090938B05E5CF4092D9
:101480008B05E2CFAE8DA1110C942313B2E0BE8F79
:10149000123089F028F4112359F0113081F08FC0F7
:1014A000163281F0103579F1133009F088C007C089
:1014B00010928C0584C0EE8DE0938C0580C0109353
:1014C0008C057DC06E317105B1F048F46431710551
:1014D00011F00C942D13F4E0F0938C0512C06832D7
:1014E000710561F06233710511F00C942D1337E032
:1014F00030938C0506C080928C0503C026E02093B3
:101500008C0581E062C040928C0559C0123129F0EF
:10151000133139F01092900502C09092900582E04C
:101520004FC082E0809390054BC06115710549F46E
:101530001A3519F410928F0502C090928F0583E03E
:1015400044C06A30710511F00C942D131A3511F452
:101550000C942D1384E039C01D3519F490928D053B
:1015600002C010928D0585E02BC0143119F49092C1
:101570008E0502C010928E0586E022C08E8D8111EC
:101580000C942313113331F41092910588E093E009
:101590009E8F1BC06A30710511F00C942D13909230
:1015A000910588E0A3E0AE8F10C0672B11F00C947A
:1015B0002D138AE00AC087E003C080E001C081E00B
:1015C000672B19F087E10C944013F30102C0EE0F72
:1015D000FF1F8A95E2F7CF019F012A213B21232B90
:1015E00009F443C085E10C944013672B59F716307A
:1015F00018F4133058F017C0183010F40C942D1351
:101600001A3000F11E3159F00C942D13123039F0BC
:101610001E3129F0111120C0909293051DC082E067
:101620008093930519C0143029F0153039F0909249
:10163000950506C082E08093950502C0109295053D
:101640008CE00BC0193021F082E08093940502C039
:10165000109294058DE001C08BE0930102C0220F2F
:10166000331F8A95E2F7C901B8CFA82AB92A29CE33
:10167000802F992787FD9095A92FB92FFC01E6545B
:10168000F109E531F10508F0E8C7EC5CFF4F0C9477
:10169000C938C0929605D0929705E0929805F092CD
:1016A000990580E07FC0C0929A05D0929B05E09298
:1016B0009C05F0929D0539A1316039A381E072C08B
:1016C000C0929E05D0929F05E092A005F092A105E0
:1016D00089A1826089A382E065C0C092A205D092F0
:1016E000A305E092A405F092A50599A1946099A3A1
:1016F00083E058C01093A60584E054C0C701B6012A
:101700000E94DF356093A7057093A8058093A90513
:101710009093AA0585E046C0C092AB05D092AC0577
:10172000E092AD05F092AE0586E03CC0C092AF05F8
:10173000D092B005E092B105F092B20587E032C0D8
:10174000C092B305D092B405E092B505F092B6050B
:1017500088E028C0C092B805D092B905E092BA05D9
:10176000F092BB05A52DA1605A2E8AE01BC0C09245
:10177000BC05D092BD05E092BE05F092BF05B52D27
:10178000B2605B2E8BE00EC0C092C005D092C10546
:10179000E092C205F092C305E52DE4605E2E8CE078
:1017A00001C089E08301082E02C0000F111F0A94B6
:1017B000E2F7980122213321232B09F046C721E6C5
:1017C00033E002C0359527958A95E2F720FF09C0DE
:1017D00020E030E0A901C701B6010E94703587FD05
:1017E00036C7202A312A6DCD552029F03E8D311182
:1017F00002C082E08E8F25FE0EC08091A7059091D9
:10180000A805A091A905B091AA0580389649A849D4
:10181000B1050CF01EC780918D05813031F4FE8D2D
:10182000F230A1F520FE1FC731C080914D05811116
:101830002DC020FE1BC080918E05813039F523E339
:1018400033E34BEC51E460919605709197058091DC
:101850009805909199050E94AE3760939605709314
:101860009705809398059093990510C080915A052B
:1018700090915B05A0915C05B0915D058093960504
:1018800090939705A0939805B093990530FC10C0EC
:101890008091560590915705A0915805B091590532
:1018A0008093B3059093B405A093B505B093B605A6
:1018B00080918B05813031F426FC02C08CE1E0C6BA
:1018C000E89426F880919005882341F0813061F0FA
:1018D00019A682E088A791E09FA30BC022E029A768
:1018E00031E038A71FA205C0A1E0A9A718A6B2E061
:1018F000BFA380918E05813021F0EE8DE33091F50C
:101900002AC0B8EBEB2EB5E0FB2E00E010E0C52CB2
:10191000D12CC601002E02C0959587950A94E2F756
:1019200080FF10C023E333E34BEC51E4D7016D910A
:101930007D918D919C910E94AE37F70160837183F8
:10194000828393830F5F1F4FF4E0EF0EF11C03308F
:101950001105F9F6D2CF80919105813019F424E078
:10196000521279C68CE0EFE6F5E0DE011D9601909B
:101970000D928A95E1F7B1FC09C030918B053F8F3C
:101980003230B9F0383009F4B0C015C180919205F9
:10199000873010F08DE174C690915205981769F365
:1019A000BE01635F7F4F0E94C222882309F465C68F
:1019B000E4CF511002C08AE163C6C1018075992746
:1019C000892B09F47BCF6091AB057091AC058091B8
:1019D000AD059091AE050E947C380E94E4356730D9
:1019E000C8F68091A605843129F0823009F035C609
:1019F00027FC33C68FEA2822662319F061506F8FC7
:101A000003C0909192059F8FBE016F5F7F4F8F8DB6
:101A10000E94C222882309F430C64090A605609037
:101A20008705709088058090890590908A05DE0171
:101A300011967D01F8EBCF2EF5E0DF2EA3E6AA2E5E
:101A4000A5E0BA2E00E010E0E52DF0E0FEA3EDA346
:101A50008DA19EA1002E02C0959587950A94E2F76C
:101A600080FF33C0F4E14F1226C0D50158962D9166
:101A70003D914D915C915B976D917D918D919C9184
:101A80000E949634F60120813181428153810E9467
:101A90009634D7016D937D938D939C931397023069
:101AA000A1F4A40193010E949634F701608371832D
:101AB000828393830AC0F60180819181A281B381E0
:101AC000F70180839183A283B3830F5F1F4FF4E0FC
:101AD000EF0EF11C24E0C20ED11C34E0A30EB11CA9
:101AE0000330110509F0B4CF0FC1552009F463CFBD
:101AF00060908705709088058090890590908A0590
:101B000008EB15E0E3E6CE2EE5E0DE2E5E018DE08B
:101B1000A80EB11CE12CF12CA52DB0E0B8A3AF8F1D
:101B20008F8D98A10E2C02C0959587950A94E2F7A7
:101B300080FF26C0F5012081318142815381D60189
:101B40006D917D918D919C910E949634F801208138
:101B50003181428153810E949634D8016D937D93E7
:101B60008D939C931397B2E0EB1214C0A4019301E0
:101B70000E949634F80160837183828393830AC044
:101B8000F601808D918DA28DB38DF80180839183B4
:101B9000A283B383FFEFEF1AFF0A0C5F1F4F24E00D
:101BA000C20ED11C34E0A30EB11C83E0E816F10490
:101BB00009F0B6CFA8C09E8D933059F4AF8DA530F3
:101BC00009F48FC0A73009F499C0A33009F09BC075
:101BD00080C0552099F340908F05809087059090A4
:101BE0008805A0908905B0908A0573E6C72E75E038
:101BF000D72E08EB15E03E01BDE06B0E711CE12C09
:101C0000F12CE52DF0E0FEA3EDA38DA19EA10E2CFD
:101C100002C0959587950A94E2F780FD0BC0F60106
:101C200080819181A281B381F80180839183A28315
:101C3000B3833EC0FF8DF730D9F1411028C0D601E3
:101C400058962D913D914D915C915B97F301608188
:101C50007181828193810E949734D8012D913D91A9
:101C60004D915C910E949734F80160837183828367
:101C70009383F2E0EF121CC0A50194010E949734F7
:101C8000D8016D937D938D939C93139711C0F601AA
:101C90002081318142815381D8016D917D918D9157
:101CA0009C910E949734F8016083718382839383AF
:101CB000FFEFEF1AFF0A24E0C20ED11C0C5F1F4F8A
:101CC00034E0630E711C83E0E816F10409F09DCF47
:101CD00075CF511001C01E8EBE016F5F7F4F86E031
:101CE00007C0511001C01E8EBE016F5F7F4F87E09D
:101CF0000E94C222882309F4C0C405C080918C05CB
:101D0000823008F0ACC41F8E10918C05183041F45D
:101D1000552009F4B3C19E8D913009F0A2C48BC245
:101D2000AE8DA23009F0AAC11123D9F020E030E035
:101D3000A901609196057091970580919805909101
:101D400099050E947035882309F48DC4143028F455
:101D5000123058F4113029F06EC2183008F44DC119
:101D60006AC2511068C21E8E8CC1552009F423CE60
:101D7000FFA1EF2FF0E0FEA3EDA338A5232F30E065
:101D80003BA72AA781E090E03C0108A402C0660CB2
:101D9000771C0A94E2F70FA002C0880F991F0A94DB
:101DA000E2F7682A792A852D90E086219721892BF0
:101DB00009F45BC4CF01880F991F880F991FFC019C
:101DC000E557FA4FDC01A45BBA4F57962D913D9130
:101DD0004D915C915A9765A576A587A590A90E941B
:101DE00096346B017C018AA59BA5880F991F880FEB
:101DF000991FFC01E557FA4FDC01A45BBA4F5796D7
:101E00002D913D914D915C915A9765A576A587A539
:101E100090A90E9496344B015C0127FE40C0E894D3
:101E200027F82091B8053091B9054091BA05509135
:101E3000BB05609163057091640580916505909183
:101E400066050E947035811120C12091BC0530913A
:101E5000BD054091BE055091BF0560916705709129
:101E600068058091690590916A050E94703581111D
:101E70000CC12091C0053091C1054091C20550911F
:101E8000C30560916B0570916C0580916D05909113
:101E90006E050E9470358111F8C081E2F1C3F9A18D
:101EA0004F2E512C64207520672809F4E0C321EFE0
:101EB000222280918E05813009F45AC00AA51BA503
:101EC000000F111F000F111F01571A4FD8011B9649
:101ED0002D913D914D915C911E97C501B4010E94D9
:101EE00096342B013C01ADA0BEA0AA0CBB1CAA0CD1
:101EF000BB1CF501E157FA4F5F0123853485458509
:101F00005685C701B6010E949634A30192010E9432
:101F10008A296B017C01D8011B962D913D914D9131
:101F20005C911E97F50163857485858596850E9471
:101F30008A294B015C016093AF057093B0058093D3
:101F4000B1059093B2059B01AC01C701B6010E9497
:101F500096346B017C01E894F7F82AE037ED43EA08
:101F60005BE3C701B6010E94733718164CF163C1D9
:101F70008AE9682E85E0782E00E010E0C201002E8C
:101F800002C0959587950A94E2F780FF10C023E37D
:101F900033E34BEC51E4D3016D917D918D919C9194
:101FA0000E94AE37F30160837183828393830F5F56
:101FB0001F4FF4E06F0E711C03301105F9F67ECF50
:101FC00020E030E040E05FE3C701B6010E947337D4
:101FD00018160CF462CF2FE632E143E85AE3C5014C
:101FE000B4010E94AE379B01AC01C701B6010E944B
:101FF000733718160CF451CF1EC1552009F4DBCCF1
:102000002091B8053091B9054091BA055091BB05B2
:1020100060916305709164058091650590916605F6
:102020000E947035811107C12091BC053091BD051A
:102030004091BE055091BF0560916705709168059C
:102040008091690590916A050E9470358111F3C0F5
:102050002091C0053091C1054091C2055091C30542
:1020600060916B0570916C0580916D0590916E0586
:102070000E947035882309F410CFDDC02E8D211108
:10208000DAC0C1018E7D9C7FD9C080918E058130E0
:10209000B1F423E333E34BEC51E46091AF0570916D
:1020A000B0058091B1059091B2050E94AE37609362
:1020B000AF057093B0058093B1059093B205409041
:1020C000AF055090B0056090B1057090B20520E06A
:1020D00030E040E850E4C301B2010E94AE37A301F2
:1020E00092010E94AE372B013C01A7019601C70166
:1020F000B6010E94AE379B01AC01C301B2010E9440
:1021000096342B013C01A5019401C501B4010E9444
:10211000AE379B01AC01C301B2010E9496342B0182
:102120003C0120E030E0A9010E94703587FDA7C284
:10213000C301B2010E943B382B013C01A50194016F
:10214000C701B6010E948A299B01AC01C301B201FB
:1021500090580E9477352B013C0180918C0583308B
:1021600021F477FA709477F870948091AF0590918C
:10217000B005A091B105B091B20589A39AA3ABA314
:10218000BCA320E030E0A901BC01CD010E94703564
:1021900087FF11C077FA709477F8709489A19AA19B
:1021A000ABA1BCA1B0588093AF059093B005A093AC
:1021B000B105B093B2050DA11EA1000F111F000FB4
:1021C000111F01571A4FA3019201C501B4010E94CA
:1021D000AE379B01AC01C701B6010E94963420E0E6
:1021E00030E040E05FE30E94AE37D8011B966D936C
:1021F0007D938D939C931E970AA51BA5000F111F1D
:10220000000F111F01571A4FA3019201C701B60118
:102210000E94AE379B01AC01C501B4010E94973406
:1022200020E030E040E05FE30E94AE37F8016387D2
:10223000748785879687C1018E7D907E892B09F0F2
:1022400018C28091A7059091A805A091A905B09109
:10225000AA0580935F0590936005A0936105B093F4
:10226000620580918D0580934D0580919605909132
:102270009705A0919805B091990580935A05909380
:102280005B05A0935C05B0935D05C090B305D0904D
:10229000B405E090B505F090B605A70196016091F0
:1022A00056057091570580915805909159050E94E7
:1022B00070358823C1F080915505882321F0B7013E
:1022C000A6010E9463138091B3059091B405A0917B
:1022D000B505B091B6058093560590935705A09328
:1022E0005805B09359058091B70580935E0580919C
:1022F000950590915505981771F0409156055091AC
:10230000570560915805709159050E94631380919B
:1023100095058093550580919405909154059817E3
:1023200031F00E94D11380919405809354058091DF
:102330008B05813051F46091AB057091AC058091B3
:10234000AD059091AE050E94D107809190058093D4
:10235000500580918E0580934E053E8D3330F9F403
:102360008091910580935105813089F48091C00559
:102370009091C105A091C205B091C30580938705D6
:1023800090938805A0938905B0938A0508C01092A0
:102390008705109288051092890510928A05809110
:1023A000920590915205981759F0809352058CE050
:1023B000FE013D96AFE6B5E001900D928A95E1F7FA
:1023C00080918F0580934F0580918B0590E0FC01F3
:1023D0003297E830F10508F04BC0E75BFF4F0C94F3
:1023E000C938BE016F5F7F4F8F8D0E94762180912B
:1023F00052059F8D89133CC08CE0FE013196AFE6FB
:10240000B5E01AC0AE8DAA2349F020E040E050E0CC
:1024100060E87FEB88EB95E00E94840420E040E0D8
:1024200050E060E87FEBCE0101960E9484048CE0CE
:10243000FE013196A3E6B5E001900D928A95E1F791
:1024400017C063E675E086E003C063E675E087E0E9
:102450000E9476210DC08CE0E8EBF5E0ABE7B5E03B
:10246000EBCF8CE0EBE7F5E0DF011D928A95E9F711
:1024700080918C0580934C05883009F498C0BE8DFE
:10248000B23009F094C090E08830910508F086C021
:10249000FC01EF5AFF4F0C94C93820E040E050E0B7
:1024A00060E87FEB0AC040915A0550915B0560914E
:1024B0005C0570915D0520914D0588EB95E00E94CB
:1024C00084046CC0C0905A05D0905B05E0905C0518
:1024D000F0905D050091AF051091B0052091B10518
:1024E0003091B20581E08F93E9A5EF93F8A5FF93B2
:1024F00015C0C0905A05D0905B05E0905C05F09047
:102500005D050091AF051091B0052091B1053091A6
:10251000B2051F9289A58F9398A59F938FA0A09035
:102520004D054AE955E068EB75E083E695E00E94C9
:10253000D2040F900F900F9031C040915A055091E6
:102540005B0560915C0570915D05E12C0AC04091CE
:102550005A0550915B0560915C0570915D05EE2414
:10256000E39400E015C040915A0550915B056091DD
:102570005C0570915D05E12C0AC040915A055091AF
:102580005B0560915C0570915D05EE24E39401E0CC
:1025900020914D0588EB95E00E9443088CE0E8EB24
:1025A000F5E0A3E6B5E001900D928A95E1F7809100
:1025B000930580935305882309F45DC00E94741627
:1025C0009091530580912C05913069F48230A1F1EE
:1025D0009FB7F894809149058860809349059FBF13
:1025E0000E94C31429C091E090934C0510925005AD
:1025F00010924F0510924D051092520510925505FC
:10260000109254058230A9F0BE01635F7F4F80E0D5
:102610000E94C222882389F18CE0FE013D96AFE63C
:10262000B5E001900D928A95E1F70E945F130E9438
:10263000C61387E00E945F2E109253051CC081E0F4
:102640001FC082E01DC088E11BC089E119C084E081
:1026500017C08BE115C085E213C084E111C08EE183
:102660000FC08FE10DC086E10BC080E209C083E29C
:1026700007C084E205C080E003C087E001C082E2B9
:10268000AB960FB6F894DEBF0FBECDBFDF91CF91F2
:102690001F910F91FF90EF90DF90CF90BF90AF9080
:1026A0009F908F907F906F905F904F903F902F9072
:1026B0000895239A259A8FE08093B30008958FE0C0
:1026C0008093B3000895CF92DF92EF92FF92CF9361
:1026D000DF931F92CDB7DEB76A017B0190912C0585
:1026E000923009F44AC089830E94E9150E94741649
:1026F0008981811104C08FE08093B3003EC0813096
:1027000011F42D9801C02D9A83E88093B000809138
:10271000B10087608093B10020E030E0A901C701DB
:10272000B6010E94703587FD11C020E030E044EB17
:1027300052E4C701B6010E947337181654F4C12C35
:10274000D12C84EBE82E82E4F82E03C0C12CD12CCE
:10275000760127E13CE641E45EE3C701B6010E9451
:10276000AE3720E030E040E751E40E9497340E9409
:102770004D360E94E4356093B3000F90DF91CF9106
:10278000FF90EF90DF90CF900895089543980895BB
:102790003B9A0C94C613823011F4439A08950C941A
:1027A000C613CF93DF931F92CDB7DEB790912C0560
:1027B000923049F089830E94741689810F90DF91CD
:1027C000CF910C94CB130F90DF91CF9108959091FE
:1027D000060180910701891708F48058891B089524
:1027E000E0ECF0E08081826080831092C50080E19F
:1027F0008093C400E1ECF0E080818061808380817F
:10280000886080838081806880830895E0910501DD
:1028100091E09E0F903409F490E02091040192130E
:1028200005C02091490524FFF8CF0895F0E0EC534E
:10283000FA4F8083909305018091C100806280935C
:10284000C10008951F920F920FB60F9211248F931B
:102850009F93EF93FF9380910401E82FF0E0EC53F6
:10286000FA4F90819093C6008F5F803409F480E026
:102870008093040190910501891305C08091C100E6
:102880008F7D8093C100FF91EF919F918F910F9069
:102890000FBE0F901F90189590910601809107012F
:1028A000891761F0E92FF0E0EC5FF94F80819F5FBD
:1028B000903809F490E09093060108958FEF089501
:1028C0001F920F920FB60F9211242F933F934F93A5
:1028D0005F936F937F938F939F93AF93BF93EF9388
:1028E000FF938091C6008F33A9F050F4883109F12D
:1028F000813211F59FB7F89480914905886015C021
:10290000803471F08E37C1F49FB7F89480914905F7
:1029100082600BC09FB7F89480914905816005C023
:102920009FB7F894809149058062809349059FBFC5
:1029300014C00E94E10811C0E091070191E09E0FD0
:10294000903809F490E020910601921731F0F0E000
:10295000EC5FF94F808390930701FF91EF91BF9156
:10296000AF919F918F917F916F915F914F913F9127
:102970002F910F900FBE0F901F9018958091070117
:10298000809306010895EF92FF920F931F93CF93C8
:10299000DF93D1E008E080E2F82E10E190E4E92E28
:1029A000C0914B05CC2389F1D0932C05C1FF02C007
:1029B00081E00FC0C2FF02C082E00BC0C3FF02C0B3
:1029C00083E007C0C4FF02C084E003C0C5FF03C0AA
:1029D00085E00E94352EC0FD08C08FB7F894909115
:1029E0004B0510924B058FBF10C081E00E945F2EF7
:1029F0009FB7F894809149058F7E809349059FBFCA
:102A00008091490584FFFCCFE8CFC0914905CC23D4
:102A100009F4C0C0C4FF04C081E080932B05D2C07C
:102A2000C0FF0AC00E9492319FB7F8948091490577
:102A30008E7F809349059FBF8C2F887609F43CC018
:102A400080912C05882349F0982F9C7769F1883074
:102A500021F40E944C1AD0932D0580912C058111F0
:102A600003C092E090932D05C6FF09C0883011F491
:102A7000E0922C0580912D05886080932D05C3FF81
:102A800005C080912C0585FF10932C05C5FF0CC057
:102A900086E00E945F2E80912D0581FDC4608460D8
:102AA00080932D05F0922C059FB7F89480914905ED
:102AB0008779809349059FBFC1FF48C08C2F8876D6
:102AC000E9F580912C05882331F08075B9F180916A
:102AD0002D0581FF33C080912D0582FF1CC08091A0
:102AE0005505882371F04091560550915705609126
:102AF0005805709159050E94C51380EA9FE00E9415
:102B00007F2980915405882331F00E94CB1388EEF1
:102B100093E00E947F290E946025892B59F08091C3
:102B20002D0583FD07C000932C050E946E1A0E949C
:102B3000851602C010922C0510922D059FB7F894AF
:102B4000809149058D7F809349059FBFC2FF22C0B8
:102B500080912C05807391F080912E0581110EC01B
:102B600080912D0582FF04C00E945F130E94C6134E
:102B700080912D05826080932D0504C010922D0553
:102B800010922C059FB7F894809149058B7F809314
:102B900049059FBF80912C058C7711F00E946E1A19
:102BA00080912C05803251F480912D0581FF06C063
:102BB0000E94C932811102C010932C0580912D050D
:102BC0008111EECEDF91CF911F910F91FF90EF9089
:102BD00008959FB7F89480914905826080934905D4
:102BE0009FBF0895CF93DF930E948E2E80912C0576
:102BF000813021F482E00E945F2E2FC00E94C932F2
:102C0000882341F0809149058062809349050E94A4
:102C1000C31402C010922C0588E091E00E94CB32D0
:102C20001CC08D3079F0DD2399F1893221F4D13047
:102C300009F04CC0D0E00E944C148F3F09F448C00A
:102C40008A3079F7EC2FF0E0E85FFE4F10820E94A7
:102C5000C31480912B05882311F0C0E0EBCF809145
:102C60000801811103C00E94E72DF7CF843229F4B7
:102C700088E091E00E94EA32F6CF80912C05813005
:102C800011F489E0F0CF88E091E00E942409EBCFB5
:102C9000813288F28F3279F28832B1F08B33B1F021
:102CA000CF3428F08BE00E94E72DC0E0C4CF2C2F5A
:102CB00030E0CF5F9FE9980FF901E85FFE4F9A314E
:102CC00008F480528083B7CFD1E0B5CFD2E0B3CF44
:102CD0000E94E9150E94C31480912B05882309F4F2
:102CE000AACFDF91CF9108950E94E9150E94C314E5
:102CF00080912B05811108C00E946025892BB1F7B6
:102D000080912C05883091F308958091C10682FF4F
:102D100002C02D9A01C02D9880912C058C70A1F0D5
:102D20008091880180939C018091890180939B010F
:102D30008091B406880F8450819580939A01809188
:102D40006F00826080936F00089580916F008D7F87
:102D500080936F0080918100887F816080938100E3
:102D6000109287018091B7068F3F21F490914B0517
:102D7000992349F090912C05943029F090E00E941D
:102D80007F2981E001C080E09091C10692FF02C0DE
:102D900091E08927882311F02D9A08952D980895A0
:102DA0001F920F920FB60F9211242F933F934F93C0
:102DB0005F936F937F938F939F93AF93BF93CF93C3
:102DC000DF93EF93FF93809187018111B7C29BB18D
:102DD00080919C01817C9E73892B8BB98BB18E7FF6
:102DE00090919B01892B8BB980919A0186BD82E0DD
:102DF00085BD81E08093870178948091AE019091A8
:102E0000AF01892B09F0A4C080918C0190918B01B6
:102E1000981709F492C0E0918C0186E0E89FF001D8
:102E20001124E055FE4FF093AF01E093AE01838192
:102E30009481909389008093880080819181909300
:102E4000AA018093A901A2818091AB018A1771F137
:102E5000A093AB0181E1A89FD0011124AC52BE4FD9
:102E6000B093AD01A093AC011D968D919D910D90F5
:102E7000BC91A02DB695A7959795879580939501C0
:102E800090939601A0939701B0939801809391013C
:102E900090939201A0939301B093940180938D013C
:102EA00090938E01A0938F01B0939001C091AC01DB
:102EB000D091AD01809188019881892780939C01F0
:102EC000258189819A81AB81BC81022E04C0B6958F
:102ED000A795979587950A94D2F780939D01909333
:102EE0009E01A0939F01B093A0018D819E81AF812F
:102EF000B885022E04C0B695A795979587950A9434
:102F0000D2F78093A1019093A201A093A301B09363
:102F1000A40189859A85AB85BC8504C0B695A79523
:102F2000979587952A95D2F78093A5019093A6014E
:102F3000A093A701B093A8010BC00E94A5169FB74C
:102F4000F894809149058460809349059FBFF6C13C
:102F50000E94CE2D10929B0180919D0190919E0127
:102F6000A0919F01B091A00140918D0150918E01DF
:102F700060918F0170919001840F951FA61FB71F5C
:102F800080938D0190938E01A0938F01B093900157
:102F9000E091AC01F091AD0145855685678570895A
:102FA000481759076A077B0708F090C021E0209373
:102FB0009B014585568567857089841B950BA60BFB
:102FC000B70B80938D0190938E01A0938F01B093E6
:102FD0009001408180912F0590913005A09131059D
:102FE000B0913205209102013091030146FF18C0D3
:102FF0000197A109B10980932F0590933005A09303
:103000003105B093320521503109121613062CF404
:10301000309303012093020119C088E090E012C0B0
:103020000196A11DB11D80932F0590933005A093AB
:103030003105B0933205C90101968930910514F02C
:1030400081E090E09093030180930201809102015E
:1030500090910301019711F480E28BB980910201F4
:1030600090910301029711F480E38BB980910201E2
:1030700090910301039711F480E18BB980910201D3
:1030800090910301049711F488E18BB980910201BA
:1030900090910301059711F488E08BB980910201AA
:1030A00090910301069711F48CE08BB98091020195
:1030B00090910301079711F484E08BB9809102018C
:1030C00090910301089711F484E28BB98091A101DA
:1030D0009091A201A091A301B091A401409191010E
:1030E000509192016091930170919401840F951F0A
:1030F000A61FB71F8093910190939201A093930113
:10310000B09394014585568567857089481759079E
:103110006A077B0708F092C020919B0121602093F1
:103120009B014585568567857089841B950BA60B89
:10313000B70B8093910190939201A0939301B09368
:10314000940140818091330590913405A09135051B
:10315000B0913605209100013091010147FF18C060
:103160000197A109B1098093330590933405A09389
:103170003505B093360521503109121613062CF48B
:10318000309301012093000119C088E090E012C043
:103190000196A11DB11D8093330590933405A09332
:1031A0003505B0933605C90101968930910514F0B3
:1031B00081E090E0909301018093000180910001F3
:1031C00090910101019711F488E088B98091000184
:1031D00090910101029711F48CE088B9809100016F
:1031E00090910101039711F484E088B98091000166
:1031F00090910101049711F486E088B98091000153
:1032000090910101059711F482E088B98091000145
:1032100090910101069711F483E088B98091000133
:1032200090910101079711F481E088B98091000124
:1032300090910101089711F489E088B98091A50166
:103240009091A601A091A701B091A801409195018C
:10325000509196016091970170919801840F951F8C
:10326000A61FB71F8093950190939601A093970195
:10327000B093980145855685678570894817590729
:103280006A077B0778F520919B01216020939B01C1
:103290004585568567857089841B950BA60BB70BF2
:1032A0008093950190939601A0939701B093980114
:1032B00020818091370590913805A0913905B09112
:1032C0003A0520FF04C00197A109B10903C0019686
:1032D000A11DB11D8093370590933805A093390542
:1032E000B0933A0580912C05843039F480914805DB
:1032F00090919B01892380939B018091A9019091DA
:10330000AA0101979093AA018093A901892B69F4DE
:103310001092AF011092AE0180918C018F5F80936B
:103320008C01863011F410928C018091890190916A
:103330009B01892780939B0110928701FF91EF9158
:10334000DF91CF91BF91AF919F918F917F916F91BD
:103350005F914F913F912F910F900FBE0F901F9053
:1033600018951F920F920FB60F9211248F93809190
:10337000890180FD589A80FF589815BC8F910F9055
:103380000FBE0F901F901895FF920F931F93CF932E
:10339000DF931092890110928801C0E0D0E00C2FD9
:1033A0001C2F2091B50630E08C2F0C2E02C03595D5
:1033B00027950A94E2F720FF07C0F09089010E9448
:1033C0000A248F29809389012091B60630E002C03B
:1033D000359527951A95E2F720FF08C010918801CE
:1033E000802F0E940C24812B809388012196C3306A
:1033F000D105A9F6DF91CF911F910F91FF9008950C
:103400000E94A5168BE2E8E5F1E0DF011D928A95A6
:10341000E9F783E2EDE8F1E0DF011D928A95E9F733
:10342000109286011092850110928C0110928B01EE
:1034300081E080938A01109287010E94C4198BB1A8
:103440008E7F90918901892B8BB98BB18E7390916E
:103450008801892B8BB90895509A259A8AB1816C7D
:103460008AB9E1E8F0E080818F7E80838081886086
:103470008083E0E8F0E080818C7F808380818F70A2
:103480008083EEE6F0E08081887F808314BC15BCE9
:103490008081816080830895CF93DF93C0918501FF
:1034A000D09186012097B9F081E080935901609115
:1034B0006F017091700180917101909172019B0177
:1034C000AC010E94AE37698B7A8B8B8B9C8B1092F0
:1034D000860110928501DF91CF9108952F923F923E
:1034E0004F925F926F927F928F929F92AF92BF9214
:1034F000CF92DF92EF92FF920F931F93CF93DF93C0
:10350000CDB7DEB7E5970FB6F894DEBF0FBECDBFDF
:1035100080912C05807709F40AC220E030E0A901EF
:1035200060916F01709170018091710190917201B1
:103530000E9470358111FBC103C680918501909175
:103540008601892B09F4FAC180918B01F6E0F89F7E
:10355000F0011124E055FE4FFE83ED838091580168
:10356000828320918501309186013E872D87D90184
:103570009596BC91BCA7F901F6A1FDA7D901979634
:10358000BC91BEA7F901F0A5FFA72091620130917F
:10359000630140916401509165016CA57DA58B2F5D
:1035A0009F2F0E94963468A779A78AA79BA720E03F
:1035B00030E0A9010E94703587FF04C018A619A643
:1035C0001AA61BA620917B01288F30917C01398F90
:1035D00040917D014A8F50917E015B8F80917301F4
:1035E0008C8F909174019D8FA0917501AE8FB091D9
:1035F0007601BF8FE0917F01E8A3F0918001F9A3EC
:10360000209181012AA3309182013BA340916B015B
:103610004CA350916C015DA380916D018EA390919C
:103620006E019FA32091770130917801409179013B
:1036300050917A0128AB39AB4AAB5BAB30916F014B
:103640003983409170014987209071013090720157
:1036500050916A015F878CA58C8B9DA59D8BAEA533
:10366000AE8BBFA5BF8B3EE3C32E33ECD32E3EE221
:10367000E32E39E3F32E188A198A1A8A1B8A260147
:103680003701EF85E111B4C3AD85BE8591962D91CB
:103690003D914D915C919497C701B6010E94AE3760
:1036A0004B015C0120E030E040E05FE30E94AE3778
:1036B0009B01AC0169817985C1010E9497349B010E
:1036C000AC01C701B6010E94AE379B01AC016C8909
:1036D0007D898E899F890E9496348B018DAB9CAB2E
:1036E000288D398D4A8D5B8D0E94703587FF86C38A
:1036F000288D398D4A8D5B8D6CA57DA58EA59FA5E6
:103700000E9496349B01AC010E9497346B017C01AE
:103710002C8D3D8D4E8D5F8D69817985C1010E9413
:1037200097349B01AC01C701B6010E9477356B014C
:103730007C0128A139A14AA15BA1688D798D8A8D70
:103740009B8D0E947035882309F455C3B1E0BF8773
:10375000FC8DF9832D8D29872E8C3F8C088D198D3A
:103760003A8D3DAB4B8D4CABA701960168897989A9
:103770008A899B890E949734688B798B8A8B9B8B73
:10378000A30192010E94703587FDF2C328A539A5D7
:103790004AA55BA5B8018DA99CA90E94733718168C
:1037A0000CF4DCC389819985D10180936F019093DA
:1037B0007001A0937101B0937201FF85F0936A01CB
:1037C00040905E0150905F016090600170906101D7
:1037D00098014DA95CA9C301B2010E94AE3769836B
:1037E0007A838B839C830E945D356B017C016091A1
:1037F0005A0170915B0180915C0190915D010E9482
:103800005D354B015C01A70196010E9496340E9430
:10381000E43569877A878B879C87E985FA85AD814E
:10382000BE81ED93FC93309709F4CDC320916601DE
:1038300030916701409168015091690168897989E7
:103840008A899B890E9497342B013C0129813A8106
:103850004B815C81C501B4010E9496349B01AC018F
:10386000C301B2010E9477354B015C0129813A8185
:103870004B815C81C701B6010E949634A501940179
:103880000E94AE3760936601709367018093680170
:103890009093690120EC31EE44E65EE4C501B40189
:1038A0000E94AE370E945D350E94E435603DB7E06E
:1038B0007B078105910508F0ACC3ED81FE8115827F
:1038C000AD81BE8114967C936E93139780918A018B
:1038D00080938B018F5F863009F4D4C380938A0173
:1038E00020916B0130916C0140916D0150916E01FE
:1038F000B8018DA99CA90E94733718160CF0C5C396
:10390000E0918501F0918601C801ADA9BCA985A30C
:1039100096A3A7A3B0A789819A81AB81BC8180932C
:103920005A0190935B01A0935C01B0935D0190916B
:103930008C0180918A01981300CE02C40E946025F8
:103940001C019093860180938501009709F4F8C3C8
:103950008091590110912C05882319F0109259017A
:10396000BEC0809158018F5F853019F08093580157
:1039700002C010925801E091580121E12E9FF00100
:103980001124EC52FE4FF0938401E0938301D101A6
:103990008C91808311964D915D916D917C911497DE
:1039A00003E0440F551F661F771F0A95D1F7418327
:1039B00052836383748315964D915D916D917C91D3
:1039C000189783E0440F551F661F771F8A95D1F71C
:1039D000458356836783708719964D915D916D91EC
:1039E0007C911C9793E0440F551F661F771F9A9593
:1039F000D1F741875287638774871D966D917D91BA
:103A00008D919C9150976B017C0123E0CC0CDD1CC7
:103A1000EE1CFF1C2A95D1F7C586D686E786F08A6C
:103A20000E94103660935A0170935B0180935C0191
:103A300090935D01F10125A136A147A150A50E94F7
:103A400077359B01AC0160935E0170935F018093B9
:103A500060019093610160E070E080EA9FE30E9462
:103A60007735609362017093630180936401909352
:103A70006501109266011092670110926801109220
:103A80006901812F8077E1F0609177017091780171
:103A90008091790190917A0160936F017093700128
:103AA00080937101909372019B01AC010E94AE372B
:103AB000D10151966D937D938D939C9354970FC034
:103AC000F10161897289838994890E943B386093EE
:103AD0006F01709370018093710190937201109245
:103AE0006B0110926C0110926D0110926E01D10168
:103AF00091968D909D90AD90BC909497A501940166
:103B000060E070E080E09FE30E9477352B013C018C
:103B10001077F101C5A0D6A0E7A0F0A4112309F405
:103B20004DC0F2E0F0936A01D10151962D913D9183
:103B30004D915C9154972D833E834F8358870E940B
:103B4000AE379B01AC01C701B6010E9496342B0130
:103B50003C0120E030E0A9010E94703587FF1DC0C4
:103B6000A5019401C501B4010E949734A7019601F3
:103B70000E94AE379B01AC016D817E818F8198855B
:103B80000E9496340E943B386093770170937801CD
:103B90008093790190937A01D7CC40926B01509237
:103BA0006C0160926D0170926E011092770110921B
:103BB00078011092790110927A01C6CC10926A01B4
:103BC000C0927B01D0927C01E0927D01F0927E0157
:103BD0000E9470254B015C0160937701709378011E
:103BE0008093790190937A019B01AC010E94AE37DA
:103BF00069837A838B839C83009185011091860170
:103C0000D80195962D913D914D915C91989729877A
:103C10003A874B875C8751962D913D914D915C91F0
:103C200054972D833E834F8358879B01AC016D8150
:103C30007E818F8198850E9496349B01AC01C301DF
:103C4000B2010E94AE379B01AC0169857A858B85F4
:103C50009C850E94973420E030E040E05FE30E94C2
:103C6000AE376B017C0120E030E0A9010E94733780
:103C700018160CF0ACC029853A854B855C85C701C8
:103C8000B6010E94703587FF8EC0F801858C968C36
:103C9000A78CB0A029813A814B815C81C501B40118
:103CA0000E9496349B01AC01C301B2010E94AE3761
:103CB00060937F01709380018093810190938201D2
:103CC000A70196010E94703587FF3DC0C501B40170
:103CD0000E943B3860937301709374018093750167
:103CE00090937601A50194016D817E818F819885E5
:103CF0000E947035811104C0F1E0F0936A0124CC78
:103D00002D813E814F815885C501B4010E949634B2
:103D10009B01AC01C301B2010E94AE379B01AC0113
:103D200060917B0170917C0180917D0190917E0179
:103D30000E94963460937B0170937C0180937D0197
:103D400090937E0101CCC0927B01D0927C01E092E5
:103D50007D01F0927E01C0927F01D0928001E092BD
:103D60008101F0928201D80191966D917D918D91A2
:103D70009C9194979B01AC010E949734A7019601F6
:103D80000E94AE3729813A814B815C810E94973431
:103D90000E943B38609373017093740180937501A6
:103DA00090937601D1CBB2E0B0936A0180916F011C
:103DB00090917001A0917101B09172018093730193
:103DC00090937401A0937501B0937601BDCB1092CE
:103DD0007B0110927C0110927D0110927E018092F5
:103DE000730190927401A0927501B0927601ACCBF0
:103DF000E13061F041C0E2E0EF87AACCA501940177
:103E000069817985C1010E9497347CC0A701960120
:103E10006C8D7D8D8E8D9F8D0E94AE379B01AC0188
:103E20006C897D898E899F890E9496348B018DAB28
:103E30009CAB28A139A14AA15BA10E94703587FFE4
:103E400093CC28A139A14AA15BA16C897D898E8977
:103E50009F890E9496342C8D3D8D4E8D5F8D0E94E2
:103E600077356B017C0108A119A15AA15DAB8BA12B
:103E70008CAB92E09F8778CCAD85BE8591962D91D5
:103E80003D914D915C919497C701B6010E94AE3768
:103E90004B015C019B01AC0169817985C1010E94E4
:103EA000733718169CF520E030E040E05FE3C50171
:103EB000B4010E94AE379B01AC0169817985C101D3
:103EC0000E9496349B01AC01C701B6010E94AE3737
:103ED0009B01AC016C897D898E899F890E949634F3
:103EE0008B018DAB9CAB2CA13DA14EA15FA10E948B
:103EF000733718165CF4A501940169817985C101B5
:103F00000E949634698379871C012ECC2CA13DA197
:103F10004EA15FA16C897D898E899F890E9496340C
:103F20009B01AC010E9497346B017C0128A939A93F
:103F30004AA95BA969817985C1010E9497349B01D7
:103F4000AC01C701B6010E9477356B017C010CA161
:103F50001DA1BEA1BDABEFA1ECAB06CC2EE333ECB3
:103F60004EE259E3C301B2010E9497342B013C0198
:103F7000288939894A895B89C301B2010E94963434
:103F80006B017C012CA13DA14EA15FA1B8018DA9BF
:103F90009CA90E94733718167CF089819985D101FC
:103FA00080936F0190937001A0937101B09372019F
:103FB0003F8530936A0104CC0C8B1D8B4DA94E8B31
:103FC0005CA95F8B5ECB80912C05807709F42ECCA9
:103FD00010926F0110927001109271011092720193
:103FE00010926601109267011092680110926901A7
:103FF000C0925A01D0925B01E0925C01F0925D01A7
:10400000A3019201C701B6010E947735AD85BE8537
:1040100070C0603AFFE07F078105910510F4E1E090
:1040200009C06034FFE17F078105910510F4E2E0EB
:1040300001C0E3E0AD81BE811596EC93AD81BE81F8
:1040400015962C911597022E04C096958795779515
:1040500067950A94D2F7E985FA8502C0EE0FFF1F33
:104060002A95E2F7ED93FC9361157105F1E08F0756
:10407000910508F425CC2FEF3FEFED81FE813483CD
:10408000238324CC10928A012BCC20E030E0A901BC
:10409000B8018DA99CA90E94733718160CF049C06D
:1040A00010926F01109270011092710110927201C2
:1040B00010926601109267011092680110926901D6
:1040C000C0925A01D0925B01E0925C01F0925D01D6
:1040D000009185011091860120915E0130915F0170
:1040E0004091600150916101C701B6010E9477358E
:1040F000D80195966D937D938D939C939897E596B3
:104100000FB6F894DEBF0FBECDBFDF91CF911F91E8
:104110000F91FF90EF90DF90CF90BF90AF909F9066
:104120008F907F906F905F904F903F902F900C9466
:10413000C52810928601109285010E944C25F7CB6C
:10414000E5960FB6F894DEBF0FBECDBFDF91CF91DD
:104150001F910F91FF90EF90DF90CF90BF90AF90A5
:104160009F908F907F906F905F904F903F902F9097
:104170000895F999FECF92BD81BD81E08FBB80B5D6
:104180000895F894F999FECF92BD81BD81E08FBB6F
:1041900040B54627842F992787FD9095262F30E03C
:1041A00082239323892B39F06F3F19F060BD84E09F
:1041B00006C084E104C0442321F060BD84E28FBBCB
:1041C000F99A789408959F92AF92BF92CF92DF921E
:1041D000EF92FF920F931F93CF93DF938C017A019D
:1041E0006B01C40ED51EEB01912C5C01A61AB70A17
:1041F000CE018A0D9B1DCC15DD0591F0911009C0F3
:10420000692D772767FD7095272F221F2227221FF0
:1042100001C021E06991922E960E0E94C120E8CF44
:10422000692DC8018E0D9F1DDF91CF911F910F91B8
:10423000FF90EF90DF90CF90BF90AF909F900C9445
:10424000C1209F92AF92BF92CF92DF92EF92FF92E6
:104250000F931F93CF93DF938B017A016C01C40EF0
:10426000D51EEC01912C5B01A81AB90AC5018C0F6F
:104270009D1FCC15DD0591F00E94B920911009C059
:10428000292D332727FD3095232F221F2227221F78
:1042900001C021E0922E980E8993E8CFC8018E0DBF
:1042A0009F1D0E94B92021E030E0981611F020E017
:1042B00030E0C901DF91CF911F910F91FF90EF90F6
:1042C000DF90CF90BF90AF909F90089521E5829F9F
:1042D000C001112440E550E09D5F0C94E32040E5CF
:1042E00050E0BC018EEA93E00C94E3202DE0829F25
:1042F000C00111244CE050E09E5F0C94E32069E083
:1043000080E090E00E94C1204DE450E064E876E057
:1043100081E090E00C94E320EF92FF920F931F93C3
:10432000CF93DF93CDB7DEB72C970FB6F894DEBFEF
:104330000FBECDBF182F80FFC1C08AE08093B406A6
:1043400089E18093B7061092B5061092B60683E015
:104350008093B8068AE097EDA3E2BCE38093B906A8
:104360009093BA06A093BB06B093BC068FE692E189
:10437000A3E0BBE38093BD069093BE06A093BF0667
:10438000B093C0061092C20680E090E0A8ECB1E4C1
:104390008093C3069093C406A093C506B093C60647
:1043A00040E050E06AEF73E44093C7065093C806BC
:1043B0006093C9067093CA068AEF90E09093CC068A
:1043C0008093CB0680E090E0A0E8BFE38093CD0629
:1043D0009093CE06A093CF06B093D0061092C1065C
:1043E00080E090E0AAE7B3E480938406909385068A
:1043F000A0938606B09387068093880690938906DB
:10440000A0938A06B0938B0680938C0690938D06BA
:10441000A0938E06B0938F0640939006509391061A
:10442000609392067093930640939406509395067A
:10443000609396067093970640939806509399065A
:1044400060939A0670939B0640E050EA6CE077E434
:1044500040939C0650939D0660939E0670939F0622
:104460004093A0065093A1066093A2067093A30602
:104470004093A4065093A5066093A6067093A706E2
:1044800040E050E068E473EC4093A8065093A9061E
:104490006093AA067093AB064093AC065093AD06AA
:1044A0006093AE067093AF064093B0065093B1068A
:1044B0006093B2067093B3060E947F2111FF10C073
:1044C000CE0101967C018CE0F70111928A95E9F703
:1044D00000E0B701802F0E9476210F5F0830C9F7F6
:1044E00012FF0AC060E080E093E00E94C12060E01B
:1044F00081E593E00E94C12013FF05C060E08EEAD1
:1045000093E00E94C1202C960FB6F894DEBF0FBE38
:10451000CDBFDF91CF911F910F91FF90EF90089544
:104520001F93CF93DF93182FEB0181E5189FB00104
:1045300011247D5F40E550E0CE010E942121892BAE
:1045400039F41882BE01812F0E94662180E001C0EB
:1045500081E0DF91CF911F910895CF93DF93EC011C
:1045600040E550E06EEA73E00E942121892B31F48E
:104570001882CE010E946F2180E001C081E0DF91AE
:10458000CF9108951F93CF93DF93182FEB018DE008
:10459000189FB00111247E5F4CE050E0CE010E94D4
:1045A0002121892B59F48CE0FE0111928A95E9F7BB
:1045B000BE01812F0E94762180E001C081E0DF9161
:1045C000CF911F91089580E090E00E94B92089303A
:1045D00059F44DE450E061E070E084E896E00E9418
:1045E000212121E0892B09F420E0822F0895CF9228
:1045F000DF92EF92FF92CF93DF93C82F6A017B0186
:1046000020E030E0A901C701B6010E94703587FDA6
:10461000E6C0C43608F445C02CE92C0F80E02330F6
:10462000B8F530E0823079F0F901EE0FFF1FEE0FA0
:10463000FF1F833011F1813019F0EC57F94F23C07F
:10464000E057F94F20C0E901CC0FDD1FCC0FDD1F73
:10465000C456D94F20E030E040E752E4C701B6012C
:104660000E94AE3720E030E040E752E40E94AE37CF
:10467000688379838A839B83AEC0E855F94FF7FA44
:10468000F094F7F8F094C082D182E282F382A3C062
:104690008F5F2A3008F4A5C0843009F4A2C02A50E4
:1046A000BECFC701B6010E947C380E94E4358C2F32
:1046B00090E08C31910508F094C0FC01E75AFF4F5F
:1046C0000C94C938633008F48EC06093B40683C07C
:1046D0006093B70680C06093B50602C06093B606CB
:1046E0000E94C41978C08091C106662311F08460CD
:1046F00007C08B7F05C08091C106662321F08064CE
:104700008093C10668C08F7BFBCF8091C106662372
:1047100011F08068F5CF8F77F3CF6093B8065BC058
:10472000C092B906D092BA06E092BB06F092BC06DF
:1047300052C0C092BD06D092BE06E092BF06F09273
:10474000C00649C08091C106662311F08160D8CFB0
:104750008E7FD6CF8091C106662321F084FF45C0AD
:104760008062CECF8F7DCCCF8091C106662311F0C1
:10477000886001C0877F8093C1060E94BB292BC03F
:104780008091C106662311F08061BACF8F7CB8CFCB
:104790006093C20620C0C092C306D092C406E092C5
:1047A000C506F092C60617C0C092C706D092C806CA
:1047B000E092C906F092CA060EC070E07093CC0673
:1047C0006093CB0608C0C092CD06D092CE06E09290
:1047D000CF06F092D0060E947F2180E007C084E0DF
:1047E00005C083E003C086E001C08AE0DF91CF917D
:1047F000FF90EF90DF90CF9008950E94E322811107
:1048000008C087E00E94E72D8FEF0E948C210C9456
:10481000962E089581E00895882321F0813021F4B7
:1048200080E8089580E4089581E00895882321F0C8
:10483000813021F484E0089582E0089580E10895B4
:104840004F925F926F927F928F929F92AF92BF92A0
:10485000CF92DF92EF92FF920F931F93CF93DF934C
:1048600010914702111101C012E11150009145024F
:10487000101709F4EFC089E2189FE0011124C75B0B
:10488000DD4F8D889E88AF88B88C69A17AA18BA1F5
:104890009CA19B01AC010E9497342DA13EA14FA188
:1048A00058A50E94AE376B017C019B01AC01B4019D
:1048B000C5010E94703587FF02C064017501A60121
:1048C000B701498B5A8B6B8B7C8B111101C012E1A4
:1048D00077247A94710E701619F029E2622E27C09F
:1048E00080914802081351C00E944C1A4EC0679C28
:1048F00080011124075B1D4F711002C092E1792ED7
:104900007A9480914802781202C00E944C1AF801F1
:10491000C588D688E788F08CA701960161897289DD
:10492000838994890E947035811106C0E8018091C5
:1049300045027812DCCF29C0F80161A172A183A1E0
:1049400094A19B01AC010E949734F80125A136A1E6
:1049500047A150A50E94AE3729893A894B895C89C5
:104960000E9497344B015C01A70196010E947035AB
:10497000F80187FF05C0818A928AA38AB48AD6CFBC
:10498000C18AD28AE38AF48AD1CF60904502F9E2E3
:104990006F9E80011124075B1D4F77247394760C62
:1049A00082E1781201C0712C5090470289E2482EB2
:1049B000751409F44DC0479CE0011124C75BDD4F1D
:1049C000F80181889288A388B488C988DA88EB883E
:1049D000FC88A7019601C501B4010E94703587FFCC
:1049E00023C0F80161A172A183A194A19B01AC0134
:1049F0000E949734F80125A136A147A150A50E9435
:104A0000AE379B01AC01C501B4010E9497344B0144
:104A10005C01A70196010E94703587FF05C0898A55
:104A20009A8AAB8ABC8A672C2D893E894F89588D1A
:104A300069897A898B899C890E947035811101C0AE
:104A4000672C7394F2E17F1201C0712C8E01B0CFFC
:104A500060924502DF91CF911F910F91FF90EF90EF
:104A6000DF90CF90BF90AF909F908F907F906F908E
:104A70005F904F9008958CE1E9E2F2E0DF011D9232
:104A80008A95E9F7109248021092470281E08093DC
:104A90004602109245020895909148028091470283
:104AA000891769F081E0890F823109F480E0209153
:104AB0004502921302C080934502809348020895F4
:104AC0008091480290914702981739F029E2829F1D
:104AD000C0011124875B9D4F089580E090E0089508
:104AE000E0914802EF5FE23109F4E0E08091470293
:104AF000E81761F089E2E89FF0011124E75BFD4FC0
:104B000061897289838994890C943B3860E070E0F4
:104B1000CB01089581E0209148029091460229132B
:104B200080E008952F923F924F925F926F927F9212
:104B30008F929F92AF92BF92CF92DF92EF92FF92AD
:104B40000F931F93CF93DF93CDB7DEB7AD970FB61B
:104B5000F894DEBF0FBECDBF142F052F6B8F7C8F57
:104B6000822E2091470239E2239F10011124F10186
:104B7000E75BFD4F1F01158616861786108A15A262
:104B800016A217A210A6108249E956E766E97EE749
:104B900041A352A363A374A35C0144E8E42E46E05E
:104BA000F42E9E01235F3F4F38A32F8F89E292E0BE
:104BB0009E8F8D8F6F01FE013196FAA3E9A3912C90
:104BC000F50161917191819191915F01F7012081CE
:104BD0003181428153810E94AE370E947E37EF8D32
:104BE000F8A16193719381939193F8A3EF8FED8D69
:104BF000FE8D4190519061907190FE8FED8F641900
:104C00007509860997092B013C0197FF07C04424C9
:104C100055243201461A570A680A790AF601418278
:104C2000528263827482F1012585368547855089D9
:104C3000421653066406750610F429013A01F10183
:104C4000458656866786708A0E941236F701208153
:104C50003181428153810E9477352B013C01E9A1CA
:104C6000FAA16193719381939193FAA3E9A320E050
:104C700030E0A9010E94703587FF0AC0F1019081E0
:104C8000892D9DA70E940C249DA5892BF10180836D
:104C9000A3019201C301B2010E94AE37F10125A127
:104CA00036A147A150A50E949734F10165A376A3D0
:104CB00087A390A79394F4E0EF0EF11C24E0C20EBA
:104CC000D11C33E093127CCF0E943B386B017C01F6
:104CD000F10165A376A387A390A785859685A7850F
:104CE000B089892B8A2B8B2B09F4FCC120E030E0A2
:104CF000A901612F702F8B8D9C8D0E94703587FDCF
:104D000021C0882061F0A7019601612F702F8B8D43
:104D10009C8D0E94AE37162F072F8B8F9C8F20E023
:104D200030E040E85FE3612F702F8B8D9C8D0E94F7
:104D3000703587FF0DC010E000E030E83B8F8FE357
:104D40008C8F06C019E906E7F6E9FB8F2EE72C8F5A
:104D5000A701960160E070E080E89FE30E9477354C
:104D600069A77AA78BA79CA7E5E3F2E0FAA3E9A3DA
:104D700020E936E038A32F8FCE010D969A8F898FC8
:104D8000FE013196FE8FED8FC12CD12C7601ED8D79
:104D9000FE8D80809180A280B38020E030E0A90168
:104DA000C501B4010E947035882309F47FC029A58C
:104DB0003AA54BA55CA5C501B4010E94AE374B01D5
:104DC0005C01ED8DFE8D60837183828393839B01F3
:104DD000AC0160E070E080E89FE30E9477352B0132
:104DE0003C01E89477F8EF8DF8A120813181428170
:104DF0005381C301B2010E94AE376BA37CA38DA384
:104E00009EA39B01AC01612F702F8B8D9C8D0E9406
:104E1000703587FF06C01BA30CA3FB8DFDA32C8D53
:104E20002EA3F101F1A1FB8FF101F2A1FC8FF101A1
:104E3000F3A1FFA3F101F4A1F8A7EF8DF8A1248558
:104E4000358546855785C301B2010E94AE373B01C7
:104E50008C019B01AC016B8D7C8D8FA198A50E946C
:104E6000703587FF04C06B8C7C8C0FA118A5C30123
:104E7000D801F10181A392A3A3A3B4A3E9A1FAA14C
:104E80002081318142815381C501B4010E94AE3736
:104E90009B01AC01C701B6010E9496346B017C01F5
:104EA0001BA10CA1FDA1FB8F2EA12C8F8D8D9E8DA2
:104EB00004969E8F8D8FE9A1FAA13496FAA3E9A3F7
:104EC0002F8D38A12C5F3F4F38A32F8FE98DFA8D9E
:104ED0008E179F0709F05BCF90914702809148029F
:104EE000981306C0F101118A128A138A148A0BC022
:104EF0002FEE3FEF4FE75FE3C701B6010E94733724
:104F0000181634F4F101118E128E138E148E5BC0BC
:104F10002FEE3FEF4FE75FEBC701B6010E947337FB
:104F2000181644F03FEEC32EDD24DA943FE7E32E5B
:104F30003FEBF32EA701960160E070E080E89FE36D
:104F40000E94963420E030E040E05FE30E94AE37FC
:104F50000E943B386B017C012091B9063091BA0662
:104F60004091BB065091BC06F10161A172A183A1E1
:104F700094A10E94AE37A70196010E94AE374B0163
:104F80005C01A701960160E070E080E89FE30E9469
:104F900096349B01AC01C501B4010E9477356B01C9
:104FA0007C0120E030E0A9010E94703587FF04C039
:104FB000C12CD12CE12CF12CA601B701F101418FBC
:104FC000528F638F748F212F302F4B8D5C8D612F0B
:104FD000702F8B8D9C8D0E94AE37162F072FF82EC9
:104FE000E92E862F902FAF2DBE2DF101858F968F44
:104FF000A78FB0A3A18CB28CC38CD48C60904102DB
:105000007090420280904302909044029301A40168
:10501000612F702F8F2D9E2D0E94703587FD0BC044
:105020009301A401B501C6010E94703587FD11C02E
:10503000530164010EC0212F302F4F2D5E2DB5017D
:10504000C6010E94703587FD04C0A12EB02ECF2C62
:10505000DE2CC501D601F101858B968BA78BB08F15
:105060008CE0FE013196A5E3B2E001900D928A95A5
:10507000E1F7812F902FAF2DBE2D809341029093A9
:105080004202A0934302B09344028CE0FE013D969D
:10509000A9E2B2E001900D928A95E1F78091460273
:1050A000809347028F5F823109F480E0809346024B
:1050B000AD960FB6F894DEBF0FBECDBFDF91CF9196
:1050C0001F910F91FF90EF90DF90CF90BF90AF9026
:1050D0009F908F907F906F905F904F903F902F9018
:1050E0000C942024AD960FB6F894DEBF0FBECDBF52
:1050F000DF91CF911F910F91FF90EF90DF90CF90B4
:10510000BF90AF909F908F907F906F905F904F90E7
:105110003F902F90089580912F0590913005A09198
:105120003105B09132058093290290932A02A09311
:105130002B02B0932C028091330590913405A091FD
:105140003505B091360580932D0290932E02A093E1
:105150002F02B09330028091370590913805A091CD
:105160003905B0913A058093310290933202A093B1
:105170003302B0933402089580914702909148021F
:10518000891708F48E5E891B08950E944C1A80913D
:105190004802809345020C9420246F927F928F9254
:1051A0009F92AF92BF92CF92DF92EF92FF920F93B6
:1051B0001F93CF93DF937C018B016A01FB018081F8
:1051C000F701E80FF11D2081EF012D3229F422961D
:1051D00021816624639407C02B3211F0219602C00E
:1051E00022962181612CA12CB12C712C60E070E001
:1051F000CB01FE0130ED932E920E29E02915C8F067
:10520000B39428E02B1588F0A1107A94A5E0B0E0C3
:105210009B01AC010E94CF38660F771F881F991F32
:10522000690D711D811D911D0BC0A11009C07394E2
:1052300007C02EEF921207C0A11005C0AA24A394A4
:1052400021962081D6CFBB2009F449C00E94103698
:105250004B015C0120E030E0A9010E9470358823F9
:1052600061F18FEF78166CF42AE037ED43E25CE3EE
:10527000C501B4010E94AE374B015C017394739475
:10528000F0CF78120BC02DEC3CEC4CEC5DE3C5018B
:10529000B4010E94AE374B015C010FC0772069F06A
:1052A00020E030E040E251E4C501B4010E94AE3795
:1052B0004B015C017A9417149CF3662021F0B7FA35
:1052C000B094B7F8B094F60180829182A282B38242
:1052D000CE19DF09C150F801C08381E001C080E030
:1052E000DF91CF911F910F91FF90EF90DF90CF90C2
:1052F000BF90AF909F908F907F906F900895009790
:1053000041F0EFE9FFE03197F1F700C000000197AD
:10531000F6CF08958F929F92AF92BF92CF92DF9275
:10532000EF92FF9269017A019B01AC010E94AE37B6
:105330004B015C01A7019601C701B6010E94AE377F
:105340009B01AC01C501B4010E949734FF90EF901E
:10535000DF90CF90BF90AF909F908F900C943B3890
:10536000EBE6F0E08081897E8083E8E6F0E08081F2
:105370008E7F8083089584B1897E84B985B18661EA
:1053800085B98091C10683FF0BC080916B00866157
:1053900080936B008091680081608093680008951D
:1053A0000C94B029CF92DF92FF920F931F93CF936B
:1053B000DF931F92CDB7DEB793B196718091C1068E
:1053C00086FD02C086E198279923D9F0C12CD12C03
:1053D000F12C01E010E08C2D99830E941624998114
:1053E000892339F098010C2C01C0220F0A94EAF7A6
:1053F000F22A8FEFC81AD80AE3E0CE16D10459F783
:1054000001C0F12C8F2D0F90DF91CF911F910F9143
:10541000FF90DF90CF9008951F920F920FB60F92DA
:1054200011242F933F934F935F936F937F938F93A9
:105430009F93AF93BF93EF93FF9380912C0581309F
:1054400071F080914B0581110AC00E94E1089FB75D
:10545000F89480914B05836080934B059FBFFF912B
:10546000EF91BF91AF919F918F917F916F915F91DC
:105470004F913F912F910F900FBE0F901F90189555
:105480002F923F924F925F926F927F928F929F9254
:10549000AF92BF92CF92DF92EF92FF920F931F9342
:1054A000CF93DF93CDB7DEB767970FB6F894DEBF23
:1054B0000FBECDBF582E80912B0581119FC128EAC8
:1054C000A22E26E0B22E9E01235F3F4F190100E07D
:1054D00010E0C12CD12C7601652C712C802F0E94FC
:1054E0000A24D1018D931D01C301002E02C09595A0
:1054F00087950A94E2F780FF1AC020E030E040EC84
:105500005FEBF50160817181828193810E94AE37EA
:10551000688B472E4C01262F372FAC01C701B601EF
:105520000E94733718161CF0C888D42C74010F5FC2
:105530001F4FF4E0AF0EB11C0330110579F68090D7
:10554000C7069090C806A090C906B090CA0624E08D
:10555000288B01E06FE275E0CE0101960E947C3459
:105560002090C206312CFE0131968FE295E09F8B90
:105570008E8B80E090E0412C10E0B701A6017058BE
:105580009301082E02C0359527950A94E2F720FF73
:1055900028C04394AE89BF891D921D921D921C9212
:1055A00013979101082E02C0359527950A94E2F7CA
:1055B00020FF03C0002319F007C0002329F0C08298
:1055C000D182E282F38204C0408351836283738379
:1055D0002DE030E02C0F3D1F280F391FD9012C91F1
:1055E000122B019634962E893F892C5F3F4F3F8BBB
:1055F0002E8B8330910521F6642D70E080E090E0E1
:105600000E9410360E943B389B01AC01C501B401D9
:105610000E94AE37AB01BC01109348054A8B5B8BEF
:105620006C8B7D8B0E948B2820E04A895B896C897A
:105630007D89CE0101960E9492250E946E1A0E94D9
:1056400085160023E9F00E94D229FE013D9620E054
:1056500030E090E06191462F412359F0AC01022ED9
:1056600002C0559547950A94E2F740FF02C0609545
:1056700016232F5F3F4F2330310561F71093480504
:105680000E946E1A809149058473C1F0809149058A
:10569000807329F00E94E1080E94C314AFC0011179
:1056A000A8C00E94D2298521A9F79FB7F8948091BC
:1056B00049058B7F809349059FBF02C010FDC1CF74
:1056C0000E94001A0E943B258091CB069091CC0647
:1056D0000E947F2931E00327C9F020E030E040EA52
:1056E00050E46091CD067091CE068091CF069091E6
:1056F000D0060E94AE376B017C018090C30690906B
:10570000C406A090C506B090C60610C0C090CD06D5
:10571000D090CE06E090CF06F090D0068090C706DD
:105720009090C806A090C906B090CA06888981509A
:10573000888B81110FCF8091C206A82FB0E0B98B62
:10574000A88BC090CD06D090CE06E090CF06F0900A
:10575000D0061601270157FA509457F8509484E860
:10576000A82E86E0B82E9FE2892E95E0992E00E0C3
:1057700010E0C301002E02C0959587950A94E2F7C8
:1057800080FF29C088899989002E02C09595879548
:105790000A94E2F7F50180FF0EC024A135A146A1CD
:1057A00057A1C701B6010E949734D5012D913D91B3
:1057B0004D915C9106C02081318142815381C201AB
:1057C000B1010E94AE370E947E37D4016D937D9364
:1057D0008D939C9313970F5F1F4FB4E08B0E911C1A
:1057E000E4E0AE0EB11C0330110519F60E948B28BF
:1057F00005C08091490582FF58CF4CCF67960FB600
:10580000F894DEBF0FBECDBFDF91CF911F910F91F6
:10581000FF90EF90DF90CF90BF90AF909F908F90D0
:105820007F906F905F904F903F902F900895BF9220
:10583000CF92DF92EF92FF920F931F93CF93DF935C
:105840008C01C8EAD6E0BB24B394F801C190D19092
:10585000E190F1908F0120E030E0A901C701B6018D
:105860000E94733718164CF0288139814A815B8178
:10587000C701B6010E94703587FDB0922E05809158
:105880002E05882361F180912C058830A9F00E94B3
:10589000E1089FB7F89480914B05856080934B0594
:1058A0009FBFDF91CF911F910F91FF90EF90DF90FD
:1058B000CF90BF900C94C3149FB7F8948091490582
:1058C0008860809349059FBF0E94C31480912B0577
:1058D00081110BC080912C058111F6CFD8CF249671
:1058E000F6E0C43BDF0709F0B0CFDF91CF911F9105
:1058F0000F91FF90EF90DF90CF90BF900895CF93DE
:10590000DF93EC018991882319F00E940614FACFE5
:10591000DF91CF910895CF93DF93FC018491EF0144
:105920002196882321F00E940614FE01F7CFDF9113
:10593000CF910895EF92FF920F931F93CF93DF9330
:105940001F92CDB7DEB7262FEDB6FEB66DB77EB788
:10595000641B71090FB6F8947EBF0FBE6DBF0DB703
:105960001EB70F5F1F4F302FF8019E2F931B941708
:1059700028F4622F0E949B389193F7CF442361F063
:10598000F801E40FF11D31978081805D49830E9409
:10599000061449814150F2CF0FB6F894FEBE0FBEF7
:1059A000EDBE0F90DF91CF911F910F91FF90EF907F
:1059B000089548E062E00C949A2C8A3020F08436F6
:1059C00020F442E003C041E001C043E06AE00C94EF
:1059D0009A2C8F929F92AF92BF92CF92DF92EF92CA
:1059E000FF920F931F93CF93DF93CDB7DEB72A9724
:1059F0000FB6F894DEBF0FBECDBF6B017C01142F34
:105A000020E030E0A9010E94703587FF07C08DE2D9
:105A10000E940614F7FAF094F7F8F094012F023080
:105A200060F020E030E048EC52E4C701B6010E948B
:105A3000AE376B017C010250F2CF10FF0AC020E0AC
:105A400030E040E251E4C701B6010E94AE376B017D
:105A50007C0120E030E040E05FE3C701B6010E9436
:105A600097340E94DF35E1E0F0E0EC0FFD1FE10F1D
:105A7000F11D2EE22083D12C5AE0852E912CA12CF1
:105A8000B12C6115710581059105A9F0D11201C0F4
:105A9000D394EE24E394F12CEC0EFD1EED0CF11CDE
:105AA000A50194010E94A738605DF7016083B901E8
:105AB000CA01D394E6CF80E3D11648F4E1E0F0E0E8
:105AC000EC0FFD1FED0DF11D8083D394F5CF8D2DCF
:105AD000D1120BC0D394D3948F5FE1E0F0E0EC0FD0
:105AE000FD1FE80FF11D80E38083DD2041F0FE0102
:105AF000ED0DF11D80810E940614DA94F6CF2A96EE
:105B00000FB6F894DEBF0FBECDBFDF91CF911F91CE
:105B10000F91FF90EF90DF90CF90BF90AF909F904C
:105B20008F9008952091C10620FF08C02BE832E431
:105B300041E25DE30E94AE3744E001C043E00C94D3
:105B4000E92C2091C10620FF08C02BE832E441E295
:105B50005DE30E94AE3741E001C040E00C94E92CC7
:105B600043E00C94E92C3D98459A08951092D10693
:105B70009091C10697FD03C090E29093D1068823CF
:105B800031F08091D10690E289278093D106089563
:105B900086B180729091D1068927089580914A0537
:105BA0008130A1F40E94C82D882381F010924A050B
:105BB0008CE0EFE2F5E0ABE3B5E001900D928A9561
:105BC000E1F7809149058064809349050895CF935A
:105BD000C82F811103C086E498E044C08EE398E0AA
:105BE0000E948B2C4C2F50E0FA013197E631F105E1
:105BF00080F5EB58FF4F0C94C93886E298E002C05C
:105C000084E198E00E948B2C2BC082E098E0FACFD0
:105C100088EF97E0F7CF87EE97E0F4CF88ED97E035
:105C2000F1CF87EB97E0EECF8EEA97E0EBCF83EAF8
:105C300097E0E8CF80E997E0E5CF82E897E0E2CF10
:105C40008CE697E0DFCF88E597E0DCCF84E497E04F
:105C5000D9CF82E397E00E948B2C8C2F0E94DD2C01
:105C60008FE297E0CF910C948B2CCF93C82F87E2D3
:105C700097E00E948B2CC33091F03CF4C13061F06E
:105C8000C230A1F481E197E00FC0C43059F0C530B3
:105C900069F487EE96E008C08CE197E005C08EEFCE
:105CA00096E002C083EF96E00E948B2C84EE96E093
:105CB0000E948B2C84EF91E0CF910C947F29CF939D
:105CC000C82F82EE96E00E948B2C8C2F90E0FC0176
:105CD0003197E830F105E8F4E557FF4F0C94C938E7
:105CE00080ED96E014C08CEB96E011C08AEA96E055
:105CF0000EC082EA96E00BC089E996E008C08EE803
:105D000096E005C086E896E002C083E796E00E9430
:105D10008B2C8FE696E0CF910C948B2C82E596E04D
:105D20000C948B2C8EE095E00C948B2CFF920F93AF
:105D30001F93CF93DF938AE095E00E948B2C809194
:105D4000B4060E94DD2C81EF94E00E948B2C8091A0
:105D5000B7060E94DD2C83ED94E00E948B2C80918D
:105D6000B5060E94DD2C8AEB94E00E948B2C80917A
:105D7000B5060E94D92C83EB94E00E948B2C809175
:105D8000B6060E94DD2C8BE994E00E948B2C80915A
:105D9000B6060E94D92C84E994E00E948B2C809155
:105DA000C10682FB882780F90E94DD2C83E794E0FE
:105DB0000E948B2C8091C10686FB882780F90E9467
:105DC000DD2C83E594E00E948B2C8091C106881F16
:105DD0008827881F0E94DD2C83E394E00E948B2C8F
:105DE0008091B8060E94DD2C8DE194E00E948B2CFE
:105DF0008091B8060E94D92C85E194E00E948B2CFA
:105E00006091B9067091BA068091BB069091BC066C
:105E10000E94B02D85EF93E00E948B2C6091BD060F
:105E20007091BE068091BF069091C0060E94B02D71
:105E30008AED93E00E948B2C8091C10681700E94B4
:105E4000DD2C8DEB93E00E948B2C8091C10685FBAD
:105E5000882780F90E94DD2C82EA93E00E948B2C37
:105E60008091C10683FB882780F90E94DD2C87E89A
:105E700093E00E948B2C8091C106829581700E94D4
:105E8000DD2C8BE693E00E948B2C8091C2060E9451
:105E9000DD2C81E593E00E948B2C8091C2060E944C
:105EA000D92C89E493E00E948B2C6091C3067091F9
:105EB000C4068091C5069091C6060E94B02D8CE262
:105EC00093E00E948B2C6091C7067091C806809168
:105ED000C9069091CA060E94B02D8FE093E00E94FF
:105EE0008B2C8091CB060E94DD2C80EF92E00E94EB
:105EF0008B2C6091CD067091CE068091CF0690914B
:105F0000D0060E94B02D87ED92E00E948B2C84E693
:105F1000F82E10E0C4E8D6E000E085ED92E00E94A3
:105F20008B2C802F8F0D0E94DD2C83ED92E00E9440
:105F30008B2C123071F01330B9F0113029F06881D8
:105F400079818A819B8117C06C857D858E859F852F
:105F500012C020E030E041E655E4688D798D8A8DED
:105F60009B8D0E94773507C08CA19DA1AEA1BFA1DA
:105F7000BC01CD0190580E94B02D80ED92E00E94AE
:105F80008B2C013029F0023031F08EEC92E005C00C
:105F90008CEC92E002C08AEC92E00E948B2C1230D2
:105FA00051F0133059F0113019F080EC92E008C034
:105FB0008EEA92E005C08DE992E002C08DE892E0A1
:105FC0000E948B2C89E892E00E948B2C0F5F249614
:105FD000033009F0A2CF8AE0F80E1F5F8CE8F812B8
:105FE00099CFDF91CF911F910F91FF900895CF939B
:105FF00083E892E00E948B2CC0E06C2F8BE395E04D
:106000000E9462340E94922DC23021F081E892E019
:106010000E948B2CCF5FC33081F78FE792E00E9404
:106020008B2C809147050E94DD2C8BE792E0CF916D
:106030000C948B2CEF92FF920F931F93CF93DF93CF
:10604000CDB7DEB72C970FB6F894DEBF0FBECDBF2D
:10605000F12CBE016F5F7F4F8F2D0E94C2228111F4
:1060600004C087E00E94E72D69C088E792E00E94A3
:106070008B2C86E0F81631F0E7E0FE1208C082E7CC
:1060800092E002C085E792E00E948B2C04C086E378
:106090008F0D0E94DD2C80E792E00E948B2C8E01F8
:1060A0000F5F1F4FE12CF8016191719181919191E6
:1060B0008F010E94922DF2E0EF1619F08EE692E029
:1060C00002C08AE692E00E948B2CE39483E0E812FF
:1060D000EACFF394E8E0FE12BCCF84E692E00E949F
:1060E0008B2C0BE715E0F12CF801619171918191F6
:1060F00091918F010E94922DF2E0FF1619F082E635
:1061000092E002C08EE592E00E948B2CF39483E033
:10611000F812EACF88E592E00E948B2C6091870507
:10612000709188058091890590918A050E94922D31
:1061300084E592E00E948B2C0E94F72F2C960FB6DC
:10614000F894DEBF0FBECDBFDF91CF911F910F91AD
:10615000FF90EF90089582E592E00E948B2C809151
:106160004C05823091F038F4882361F08130A9F435
:106170008CE492E00CC0833069F0883071F482E4E2
:1061800092E005C08FE492E002C089E492E00E94B0
:106190008B2C0CC086E492E0FACF8DE392E00E9453
:1061A0008B2C80914C0582500E94DD2C8AE392E07A
:1061B0000E948B2C809152058A5C0E94DD2C80917C
:1061C0005005813049F028F0823051F48BE292E0A2
:1061D00005C085E392E002C080E392E00E948B2C30
:1061E00080914E05811103C086E292E002C081E2F7
:1061F00092E00E948B2C80914F05811103C08CE1AD
:1062000092E002C087E192E00E948B2C80914D05C4
:10621000813019F482E192E002C08DE092E00E94A8
:106220008B2C80915305813049F028F0823051F455
:1062300081E092E005C089E092E002C085E092E052
:106240000E948B2C80915505813031F040F08230D6
:1062500051F489EF91E005C08DEF91E002C085EF28
:1062600091E00E948B2C80915405882329F0823084
:1062700039F48DEE91E002C081EF91E00E948B2C09
:106280008AEE91E00E948B2C80915E050E94DD2CAD
:1062900087EE91E00E948B2C60915A0570915B050E
:1062A00080915C0590915D050E94A12D84EE91E0A6
:1062B0000E948B2C6091560570915705809158056E
:1062C000909159050E94A12D80EE91E00C948B2CA9
:1062D0001F93CF93DF93182FEB018DED91E00E9478
:1062E0008B2C812F0E94DD2C8BED91E00E948B2C5A
:1062F000CE010E947F2C88ED91E0DF91CF911F911C
:106300000C948B2CCF93DF93EC0188EC91E00E94EE
:106310008B2CCE010E947F2C84EC91E0DF91CF91F9
:106320000C948B2CBF92CF92DF92EF92FF920F933F
:106330001F93CF93DF93CDB7DEB768970FB6F8946E
:10634000DEBF0FBECDBF8CE0EFE2F5E0DE011D96B3
:1063500001900D928A95E1F780912C058430E9F047
:1063600040F48130E9F080F0823009F58FE991E066
:106370001CC0803179F018F4883049F018C08032A0
:1063800091F0803421F013C08EEB91E00EC089EBC8
:1063900091E00BC083EB91E008C08DEA91E005C06D
:1063A00086EA91E002C089E991E00E948B2C8091FD
:1063B000B806837039F0BE01635F7F4FCE0101964E
:1063C0000E947C348091B80680FD05C08091B8069B
:1063D00081FF6DC01FC082E991E00E948B2C698112
:1063E0007A818B819C810E94922D80E991E00E94AC
:1063F0008B2C6D817E818F8198850E94922D80E902
:1064000091E00E948B2C69857A858B859C850E9402
:10641000922DDCCF89E891E00E948B2C9FE6E92E3B
:1064200095E0F92E8E010F5F1F4FB12C6801F70127
:1064300061917191819191917F0120853185428592
:1064400053850E9497349B01AC01F80160817181F2
:10645000828193810E949634F801608371838283E4
:106460009383F2E0BF120FC0209187053091880519
:106470004091890550918A050E949634F801608305
:106480007183828393830C5F1F4FF601608171815A
:10649000828193810E94922DF2E0BF1621F087E85D
:1064A00091E00E948B2CB39423E0B212BFCF809175
:1064B000B80682FF08C081E891E00E948B2C0E9400
:1064C000BC280E94DD2C8091B80683FF08C08CE7B1
:1064D00091E00E948B2C0E94E7130E94DD2C80919A
:1064E000B80684FF0AC086E791E00E948B2C0E94C8
:1064F000D22943E062E00E949A2C82E791E00E9458
:106500008B2C68960FB6F894DEBF0FBECDBFDF911F
:10651000CF911F910F91FF90EF90DF90CF90BF90A0
:1065200008953E98469AECE6F0E08081806480838E
:10653000E8E6F0E080818260808308951F920F92E8
:106540000FB60F9211242F933F934F935F936F9346
:106550007F938F939F93AF93BF93EF93FF9386B1F6
:106560008095982F907486FF03C091110E94E108D6
:10657000FF91EF91BF91AF919F918F917F916F911B
:106580005F914F913F912F910F900FBE0F901F90F1
:10659000189580E008951F93CF93DF93EC0110E0EE
:1065A000BE01812F0E949022811102C087E009C0A4
:1065B0008881882341F0CE010E947F2CCE010E9469
:1065C00024090E94E72D1F5F123051F7DF91CF9110
:1065D0001F9108958F929F92AF92BF92CF92DF92B8
:1065E000EF92FF921F93CF93DF93CDB7DEB729973A
:1065F0000FB6F894DEBF0FBECDBF7C0181E0898766
:10660000F7018181833479F034F4882349F08432AE
:1066100009F040C008C0873431F08835D9F503C08F
:106620000E94922E1AC0F7019281911138C18334D1
:10663000B1F01CF4843231F010C0873461F0883539
:10664000F9F00BC080912C05887111F088E028C109
:106650000E94962E02C00E94AB3080E021C1809142
:106660002C05823021F40E94E10885E006C08111EA
:10667000EDCF82E080932C0584E00E945F2EEDCF69
:1066800080912C05813049F783E00E945F2E1092A3
:106690002C05E3CF90912C059230C0F6893459F146
:1066A0002CF4833251F0883489F08AC08E3409F496
:1066B0006AC0823509F440C083C082E08987F7014F
:1066C00082818111ECC00E941A30C7CF8091C1062F
:1066D00084FFE3C084E080932C050E943008809101
:1066E0002B058111BACF10922C050E94A516C70167
:1066F0000E94CB32B2CF82E08987F701828181117B
:1067000007C0C7010E94AD22C7010E948231A5CFF8
:106710008D3309F0C4C083E0F701E80FF11D9081CB
:10672000DF0113979C938F5F90819111F5CF89873B
:10673000C7010E946F2191CFF7018281833509F053
:10674000AEC08381843509F0AAC084818D3309F0FD
:10675000A6C086818111A3C085E0898785818432A6
:1067600039F08A3239F0833209F099C082E003C0EF
:1067700081E001C08FEF0E948C2188E00E945F2E93
:106780000E94E1086ACF82E08987F7018281811146
:1067900013C010E0B701812F0E949022811104C024
:1067A00087E00E94E72D04C0B701812F0E94683165
:1067B0001F5F123079F751CF911148CF11E001C01E
:1067C00010E0AE014B5F5F4FBE01675F7F4FC701B7
:1067D0000E94CD28811102C082E062C0898521E03B
:1067E000280F2987F701E80FF11D80818D3309F00B
:1067F00056C0112321F1822F90E0E22FF0E0D70163
:10680000AE0FBF1F3C91E81BF90BEE0DFF1D30834F
:106810002F5F3C913111F1CF2987C7010E942409D4
:1068200081113EC06D817E818F8198850E947C3868
:106830000E94E435862FB7010E9466210ECFAE017B
:106840004F5F5F4FBE01675F7F4FC7010E94CD283A
:10685000882311F28985F701E80FF11D80818111EC
:106860001EC0CD80DE80EF80F88420E030E04FE76E
:1068700053E4C701B6010E947337181684F089806B
:106880009A80AB80BC80C701B6010E94E435862F98
:10689000B501A4010E94F72203C085E001C083E096
:1068A00029960FB6F894DEBF0FBECDBFDF91CF9112
:1068B0001F91FF90EF90DF90CF90BF90AF909F908F
:1068C0008F900895CF93DF9324E0629FE00111241D
:1068D0008C0F9D1FFC0160817181828193810E94D8
:1068E0001236CC57D94F288139814A815B810E9469
:1068F0007735DF91CF910895FF920F931F93CF9338
:10690000DF938B01EC01F12C6F2DC8010E946234E2
:106910006993799389939993F39483E0F812F4CF70
:10692000DF91CF911F910F91FF9008955058BB2791
:10693000AA270ED076C23FD230F044D220F031F4F4
:106940009F3F11F41EF40FC20EF4E095E7FBDCC18B
:10695000E92F89D280F3BA17620773078407950776
:1069600018F071F49EF5B8C20EF4E0950B2EBA2F14
:10697000A02D0B01B90190010C01CA01A001112445
:10698000FF27591B99F0593F50F4503E68F11A16F1
:10699000F040A22F232F342F4427585FF3CF469582
:1069A00037952795A795F0405395C9F77EF41F16A4
:1069B000BA0B620B730B840BBAF09150A1F0FF0F6E
:1069C000BB1F661F771F881FC2F70EC0BA0F621F5A
:1069D000731F841F48F4879577956795B795F7954A
:1069E0009E3F08F0B3CF9395880F08F09927EE0FDC
:1069F000979587950895DFD158F080E891E009F4E4
:106A00009EEFE0D128F040E851E059F45EEF09C074
:106A1000AAC162C2E92FE07826D268F3092E052ABE
:106A2000C1F3261737074807590738F00E2E07F825
:106A3000E02569F0E025E0640AC0EF6307F8009400
:106A400007FADB01B9019D01DC01CA01AD01EF9339
:106A50005DD0E7D10AD05F91552331F02BED3FE0B7
:106A600049E450FD49EC63CF0895DF93DD27B92F4A
:106A7000BF7740E85FE31616170648075B0710F478
:106A8000D92F35D29F938F937F936F9332D3E6E2C2
:106A9000F1E06CD1C6D12F913F914F915F916AD2B5
:106AA000DD2349F09058A2EA2AED3FE049EC5FE38C
:106AB000D0785D274DDFDF91B4C1F7D180F09F37EB
:106AC00040F491110EF409C260E070E080E89FE3A9
:106AD000089526F01B16611D711D811D1BC135C156
:106AE000EFD008F481E0089575D1E395ABC10CD0E7
:106AF00098C168D140F05FD130F021F45F3F19F0C8
:106B000003C15111EAC12FC1AED198F39923C9F342
:106B10005523B1F3951B550BBB27AA2762177307A3
:106B2000840738F09F5F5F4F220F331F441FAA1F57
:106B3000A9F333D00E2E3AF0E0E830D09150504017
:106B4000E695001CCAF729D0FE2F27D0660F771FC5
:106B5000881FBB1F261737074807AB07B0E809F0A7
:106B6000BB0B802DBF01FF2793585F4F2AF09E3F3C
:106B7000510568F0C9C0B1C15F3FECF3983EDCF34A
:106B8000869577956795B795F7959F5FC9F7880FB5
:106B9000911D9695879597F90895E1E0660F771F07
:106BA000881FBB1F621773078407BA0720F0621B98
:106BB000730B840BBA0BEE1F88F7E095089504D091
:106BC0006894B1118AC1089556D188F09F5790F00A
:106BD000B92F9927B751A0F0D1F0660F771F881F02
:106BE000991F1AF0BA95C9F712C0B13081F074D16B
:106BF000B1E0089571C1672F782F8827B85F39F009
:106C0000B93FCCF3869577956795B395D9F73EF460
:106C100090958095709561957F4F8F4F9F4F089508
:106C2000E89409C097FB3EF4909580957095619526
:106C30007F4F8F4F9F4F9923A9F0F92F96E9BB27DC
:106C40009395F695879577956795B795F111F8CF58
:106C5000FAF4BB0F11F460FF1BC06F5F7F4F8F4FC3
:106C60009F4F16C0882311F096E911C0772321F0B9
:106C70009EE8872F762F05C0662371F096E8862F51
:106C800070E060E02AF09A95660F771F881FDAF7A8
:106C9000880F9695879597F9089507D180F09F37CB
:106CA00040F491110EF019C160E070E080E89FEBB4
:106CB000089526F41B16611D711D811D2BC045C052
:106CC000990F0008550FAA0BE0E8FEEF16161706FD
:106CD000E807F907C0F012161306E407F50798F065
:106CE000621B730B840B950B39F40A2661F0232B7E
:106CF000242B252B21F408950A2609F4A140A695FA
:106D00008FEF811D811D089597F99F6780E870E0DE
:106D100060E00895882371F4772321F09850872B41
:106D2000762F07C0662311F499270DC09051862B4A
:106D300070E060E02AF09A95660F771F881FDAF7F7
:106D4000880F9695879597F908959F3F31F0915058
:106D500020F4879577956795B795880F911D96953F
:106D6000879597F908959FEF80EC0895DF93CF936F
:106D70001F930F93FF92EF92DF927B018C01689437
:106D800005C0DA2EEF01F6D0FE01E894A591259119
:106D9000359145915591AEF3EF01DADDFE01970192
:106DA000A801DA9479F7DF90EF90FF900F911F918F
:106DB000CF91DF91089500240A941616170618063D
:106DC0000906089500240A941216130614060506EF
:106DD0000895C9CF50D0E8F3E894E0E0BB279F576F
:106DE000F0F02AED3FE049EC06C0EE0FBB0F661F46
:106DF000771F881F28F0B23A62077307840728F0CC
:106E0000B25A620B730B840BE3959A9572F7803834
:106E100030F49A95BB0F661F771F881FD2F79048F2
:106E200096CF092E0394000C11F4882352F0BB0F67
:106E300040F4BF2B11F460FF04C06F5F7F4F8F4F92
:106E40009F4F0895EF93E0FF06C0A2EA2AED3FE0CE
:106E500049EC5FEB7DDDE5DF0F90039401FC90587A
:106E6000E3E5F1E057C157FD9058440F551F59F025
:106E70005F3F71F04795880F97FB991F61F09F3F27
:106E800079F087950895121613061406551FF2CF50
:106E90004695F1DF08C0161617061806991FF1CFA0
:106EA00086957105610508940895E5DFA0F0BEE7B9
:106EB000B91788F4BB279F3860F41616B11D672FE9
:106EC000782F8827985FF7CF869577956795B11DBE
:106ED00093959639C8F30895E894BB2766277727DA
:106EE000CB0197F90895ECDE08F48FEF08959B012C
:106EF000AC0160E070E080E89FE3F9CDBCDF58F1C1
:106F00009E5758F19851A0F0E9F0983020F5092EDD
:106F10009927660F771F881F991F0A94D1F712C00F
:106F2000062E672F782F8827985F11F4000C07C072
:106F3000993FB4F38695779567959395D9F7611D39
:106F4000711D811D3EF490958095709561957F4FE0
:106F50008F4F9F4F08956894C0CFBECF0BD061CFA5
:106F60002ADF28F02FDF18F0952309F0CDCEFBCED5
:106F70001124B3CF78DFA0F3959FD1F3950F50E0A4
:106F8000551F629FF001729FBB27F00DB11D639FDB
:106F9000AA27F00DB11DAA1F649F6627B00DA11D81
:106FA000661F829F2227B00DA11D621F739FB00D27
:106FB000A11D621F839FA00D611D221F749F332797
:106FC000A00D611D231F849F600D211D822F762F30
:106FD0006A2F11249F5750408AF0E1F088234AF02D
:106FE000EE0FFF1FBB1F661F771F881F9150504079
:106FF000A9F79E3F510570F087CE6FCF5F3FECF34E
:10700000983EDCF3869577956795B795F795E79564
:107010009F5FC1F7FE2B880F911D9695879597F975
:10702000089529DFE0F09E37D8F09639B8F49E38FD
:1070300048F4672F782F8827985FF9CF8695779542
:10704000679593959539D0F3B62FB1706B0F711D7D
:10705000811D20F487957795679593955BCE75CEC6
:107060003CCF9F93B7DE0F9007FCEE5FEBCE11F4A1
:107070000EF479CE6ACEFFDED0F39923D9F3CEF3A6
:107080009F57550B87FF3FD00024A0E640EA9001B0
:1070900080585695979528F4805C660F771F881F57
:1070A00020F026173707480730F4621B730B840B58
:1070B000202931294A2BA69517940794202531259C
:1070C0004A2758F7660F771F881F20F026173707C3
:1070D000480730F4620B730B840B200D311D411DEA
:1070E000A09581F7B901842F9158880F96958795BF
:1070F00008959B01AC0132CFD8DE20F09F3708F411
:10710000ECCE08CE22CE91505040660F771F881FDC
:10711000D2F708959F938F937F936F93FF93EF938D
:107120009B01AC011BDFEF91FF9120DE2F913F917E
:107130004F915F9113CF991B79E004C0991F961767
:1071400008F0961B881F7A95C9F780950895A1E2EB
:107150001A2EAA1BBB1BFD010DC0AA1FBB1FEE1FD1
:10716000FF1FA217B307E407F50720F0A21BB30B1C
:10717000E40BF50B661F771F881F991F1A9469F798
:1071800060957095809590959B01AC01BD01CF01F4
:107190000895EE0FFF1F0590F491E02D09940E94D1
:1071A000DA38A59F900DB49F900DA49F800D911D7E
:1071B00011240895A29FB001B39FC001A39F700D39
:1071C000811D1124911DB29F700D811D1124911DEF
:0671D0000895F894FFCFC2
:0471D60001000100B3
:00000001FF
